:100000000C94BF020C94F7020C94F7020C94F702C4
:100010000C94F7020C94F7020C94F7020C94F7027C
:100020000C94F7020C94F7020C94CA310C949C3295
:100030000C948D2C0C94F7020C94F7020C94F7029C
:100040000C94F7020C94F7020C94F7020C94F7024C
:100050000C94F7020C94312D0C94F7020C94F702D7
:100060000C94F7020C94F7020C94F7020C94F7022C
:100070000C94F7020C94F7020C94F7020C94F7021C
:100080000C94F7020C94F7020C94F7020C94F7020C
:100090000C94F7020C94F7020C94F7020C94F702FC
:1000A0000C94F7020C94F7020C94F7023A053A0507
:1000B00066056605CE05EC0504070407F7059006FE
:1000C000A106A106093330332834303328347C3379
:1000D0009F332834F6330534009B8B7B00AB8A7A40
:1000E00000AA9A7900A9998900A8988800A79787FB
:1000F00000A6968600A5958500A49484003C4C5CDF
:10010000002C4D5D002D3D5E002E3E4E00304050D7
:1001100000314151002A3A4A00293949002838481B
:10012000002737470026364600253556002445551A
:100130000034445400AC9C8C00AD9D8D00AE9E8E6E
:1001400000AF9F8F00B0A09000B1A1910032425249
:10015000002B3B4B01A9998901A8988801A7978793
:1001600001A6968601A5958501A49484013C4C5C6A
:10017000012C4D5D012D3D5E012E3E4E012F3F4F66
:10018000013040500033435301AB8A7A012838488C
:1001900001273747012636460125355601244555A6
:1001A00001AC9C8C01AD9D8D01AE9E8E01AF9F8FE9
:1001B00001314151013242520133435300B2A28115
:1001C000019B8B7B012B3B4B012A3A4A013444545F
:1001D00001B1A19101B2A28101B3928201A39383E3
:1001E00000A3938300B39282165C1E001F002000C0
:1001F00021002200230024002500260027002D00D6
:100200002E002A004A002B0014001A0008001500D6
:1002100017001C0018000C00120013002F00300003
:1002200031004B00396104001600070009000A0084
:100230000B000D000E000F003300340000002800FA
:100240004E00E1001D001B00060019000500110012
:100250001000360037003800E500000052004D0065
:10026000E000E300E200000000002C0000000000BD
:10027000E6000151E4005000000051004F00165C00
:100280003A003B003C003D003E003F004000410082
:1002900042004300440045004C004A000100C35C9A
:1002A000C45CC65CC75CC85CC95CCA5CCB5C010052
:1002B000460047004800005C4B003961CC5CCD5CD7
:1002C0000100010001000100010001000100010026
:1002D00001000000DF5C4E00E100010001000100B0
:1002E00001000100145C0100010001000100010097
:1002F0000000A900A80001000100010000000000AA
:10030000010000000000010001000100AC0000003D
:10031000AA00AB000001010101010101010102027B
:1003200002020202020202030303030303030304A3
:10033000040404040404050505050506060606066E
:10034000070707070708080808090909090A0A0A28
:100350000B0B0B0C0C0C0D0D0D0E0E0E0F0F0F10CA
:100360001011111112121313141415151616171754
:10037000181819191A1A1B1B1C1D1D1E1E1F2020C0
:10038000212222232424252626272829292A2B2C0A
:100390002D2D2E2F30313232333435363738393A2D
:1003A0003B3C3D3E3F404142434445464748494A25
:1003B0004C4D4E4F50515354555658595A5B5D5EF3
:1003C0005F616264656668696B6C6D6F707273758E
:1003D00077787A7B7D7E8082838587888A8C8E8FF2
:1003E00091939596989A9C9EA0A2A3A5A7A9ABAD20
:1003F000AFB1B3B5B7BABCBEC0C2C4C6C9CBCDCF0E
:10040000D1D4D6D8DBDDDFE2E4E7E9EBEEF0F3F5BB
:10041000F8FAFDFF100344005A0036003500520080
:100420004700420000000E0344005A0054004500FB
:100430004300480000000403090409023B000201D4
:1004400000A0FA09040000010301010009211101C3
:100450000001224000070581030800010904010092
:10046000010300000009211101000122B600070567
:10047000820320000112010002000000085A4421FA
:100480001402000102000105010902A1018502090F
:1004900001A1000509190129081500250195087514
:1004A0000181020501093009311581257F95027509
:1004B00008810609381581257F9501750881060593
:1004C0000C0A38021581257F950175088106C0C088
:1004D00005010980A101850319012AB7001501262C
:1004E000B700950175108100C0050C0901A10185B7
:1004F0000419012AA002150126A002950175108198
:1005000000C005010906A1018506050719E029E7D4
:10051000150025019508750181020507190029EFCD
:100520001500250195F075018102050819012905BD
:10053000950575019102950175039101C0050109A9
:1005400006A101050719E029E715002501950875A1
:100550000181029501750881010507190029FF1520
:100560000026FF0095067508810005081901290578
:10057000950575019102950175039101C000112443
:100580001FBECFEFDAE0DEBFCDBF04B603FE18C05A
:100590008091DC069091DD06A091DE06B091DF0629
:1005A0008730904BA740B04B59F41092DC06109264
:1005B000DD061092DE061092DF06E0E0F8E3099512
:1005C00012E0A0E0B1E0E8E7FBE602C005900D9282
:1005D000A63CB107D9F726E0A6ECB2E001C01D9217
:1005E000AC3DB207E1F70E9419130C94BA350C9494
:1005F00000000E943D2B81FF07C02FEF4FEF6FEFF0
:100600008EE190E00C942619089581E0089581E030
:1006100008950C94070308950C940B031F93CF9334
:10062000DF9300D000D01F92CDB7DEB749835A8345
:100630006B833091C90289819A81311114C066237C
:1006400059F0222349F00E944109182F682F89810F
:100650009A810E94EA0803C00E941509182F698137
:100660007A81812F04C00E94410969817A810F90AB
:100670000F900F900F900F90DF91CF911F910C94DE
:100680008410FC01262F4081518162817381848115
:100690000C940E0381E00895CF93DF93EC0160E0AA
:1006A0000E944103BE01DF91CF910C940C030C9486
:1006B000CA110C94C61108950E9494070E945B030E
:1006C0002FEF84E39CE0215080409040E1F700C090
:1006D00000000C94572D0F931F93CF93DF938C0141
:1006E00061E00E944103EC01B8010E9409038823E4
:1006F00009F444C0B801CE010E94F7298823F1F122
:10070000B801CE010E940B288823C1F1B801CE01A7
:100710000E945329882391F1B801CE010E946E27CF
:10072000882361F1F8018281882309F1CB358DE5B9
:10073000D807C1F050F4C115FCE5DF0781F0CF3DCB
:10074000DC45A9F40E94780E19C0CC35EDE5DE0732
:1007500061F0CD35DD4559F40E94BB0D08C00E9403
:100760005C030CC00E94C40D02C00E94C70DC801EA
:10077000DF91CF911F910F910C94050380E0DF91E1
:10078000CF911F910F9108950E946F2C0E94182302
:100790000E94E50381E00C9417240E94E80380E0A6
:1007A0000E9417240C94752C08950C94D40381E0B6
:1007B00008950C94D7030895CF93C82F0E94D503B2
:1007C0008C2F0E94D903CF91089580E00C94DC0314
:1007D0000E94312B0C94DC030E94312B9091C802B3
:1007E000891721F08093C8020C94DC030895CF93FD
:1007F000DF93CDB7DEB72B970FB6F894DEBF0FBEF1
:10080000CDBF4F83588769877A878B8761110E9494
:10081000070D9E012F5F3F4F86E0F90111928A95E7
:10082000E9F785E0FE013796D90101900D928A958E
:10083000E1F789819A814C815D81452B31F09F3FA1
:1008400031F491E08F3F19F403C091E001C090E0D2
:1008500090FF09C049815A816B817C818D819E8185
:100860000E94280C05C0C9010E944A038111F2CFE1
:100870002B960FB6F894DEBF0FBECDBFDF91CF91A0
:100880000895FC01808191810E9483090895CF938E
:10089000882309F450C0C82F8CEF8C0F813AD0F414
:1008A0006C2F80911D0290911E020E94AA2B88231A
:1008B00049F06C2F80911D0290911E020E94352CF0
:1008C0000E94290D6C2F80911D0290911E020E94A2
:1008D0002A2C0CC080E28C0F883058F4C77081E05D
:1008E00001C0880FCA95EAF70E94EA0CCF910C94D8
:1008F000290DEBE5EC0FE33040F4F0E0E359FD4F58
:10090000808190E0CF910C94682BE8E5EC0FE73103
:1009100050F4F0E0EE0FFF1FE15CFD4F808191810C
:10092000CF910C947E2BCD3E30F08C2F0E949E13E5
:10093000CF910C947014CF910895882389F19CEF86
:10094000980F913A40F4682F80911D0290911E02F9
:100950000E94352C0DC090E2980F983058F48770A3
:1009600091E001C0990F8A95EAF7892F0E94F00C57
:100970000C94290D9BE5980F933020F480E090E0D3
:100980000C94682B98E5980F973120F480E090E064
:100990000C947E2B8D3E20F00E94F9130C94701461
:1009A00008951F93CF93DF93182FEB010E94470404
:1009B000209741F08FE99FE00197F1F700C0000018
:1009C0002197F6CF812FDF91CF911F910C949D0439
:1009D000893319F060E070E002C060E570E00C94CB
:1009E000D104882321F00E94EA0C0C94290D08956B
:1009F000882321F00E94F00C0C94290D0895CF92C9
:100A0000DF92EF92FF920F931F93CF93DF937C01BE
:100A1000D62FC72FFC011281058102950F700E940D
:100A2000E00C8823B9F01123A9F08C2F807F80344B
:100A300021F080E28D0F883068F080914F0582FDB3
:100A400009C082E00E94890D0E94E00C91E0D82E3E
:100A5000D92601C0D12CCC2EC2948FE0C8228C2D77
:100A600090E08C30910508F0CFC1FC01EA5AFF4FAD
:100A70000C94C5348C2F807FCF70882311F0C295E1
:100A8000C07F112399F0CC2309F4AAC180E28D0F15
:100A9000883010F0D11104C08C2F0E94EA0C03C0E2
:100AA0008C2F0E94FA0C0E94290D9AC18D2F0E9452
:100AB0009D04CC2309F4A8C180E28D0F883038F161
:100AC000DD2329F18C2F0E94000D24C08C2F807F04
:100AD000CF70803211F0C295C07FDD2319F0D13084
:100AE000A1F13DC080914F0582FF17C0112349F04D
:100AF000CC2329F08C2F0E94EA0C0E94290D80E063
:100B000070C180E00E949D04CC2309F47DC18C2F2C
:100B10000E94F00C0E94290D77C1112371F000236F
:100B200041F0013031F40E940A0D8C2B0E94120D0D
:100B30006BC10E940A0D8C2B1DC0002319F00130DF
:100B400009F462C10E941F0D25C0112321F0063057
:100B500008F05AC10EC0053008F056C11BC0112361
:100B600061F0002331F0F701858180FF39C18F707A
:100B700085838C2F0E94F10447C1002359F0D9339B
:100B800009F03FC1FFEF07EE13E0F15000401040C5
:100B9000E1F735C18C2F0E94F80436C18C2F869561
:100BA0008695837019F0813061F02EC1112321F0F8
:100BB0008D2F9C2F937002C080E090E00E94682BE4
:100BC0002BC1112321F08D2F9C2F937002C080E048
:100BD00090E00E947E2B20C18D2F112319F00E94DE
:100BE0009E1302C00E94F9130E94701415C18C2F2D
:100BF000837009F047C011110BC12D2F2295269546
:100C00002770220F220F6D2F6F70862F90E0A0E0CB
:100C1000B0E0022E04C0880F991FAA1FBB1F0A94C0
:100C2000D2F7D4FF10C04FE050E060E070E004C0A5
:100C3000440F551F661F771F2A95D2F74095509590
:100C40006095709503C040E050E0BA01C695C69526
:100C5000C3708A019B01082B192B2A2B3B2BC9013E
:100C6000B801C23049F058F4C13019F00E940008B0
:100C7000CFC00E94EE07CCC00E941208C9C00E94DB
:100C8000EC07C6C0112319F08C2F817001C0869526
:100C9000882309F4BDC02D2F229526952770220F99
:100CA000220F6D2F6F70862F90E0A0E0B0E0022E33
:100CB00004C0880F991FAA1FBB1F0A94D2F7D4FF44
:100CC00010C04FE050E060E070E004C0440F551FDA
:100CD000661F771F2A95D2F74095509560957095BD
:100CE00003C040E050E0BA01C695C695C3708A01C2
:100CF0009B01082B192B2A2B3B2BC901B801C230B1
:100D000049F058F4C13019F00E94C50881C00E9412
:100D1000B3087EC00E94D7087BC00E94260878C016
:100D2000CF70112339F08C2F0E944C088D2F0E9418
:100D3000F1046EC08D2F0E94F8048C2F0E946D0864
:100D400067C0D23F21F128F4D03F41F0D13FC1F03C
:100D500043C0D33F19F1D43F79F03EC0112341F095
:100D6000053008F051C08C2F8F710E9492084CC042
:100D7000063008F049C0F7CF80914F0582FF18C0B8
:100D8000112339F08C2F8F710E944C083DC0112324
:100D9000C9F38C2F8F710E946D0836C0112329F082
:100DA0008C2F8F710E9437082FC00E9432082CC0F0
:100DB000112349F0CF718C2F0E944C0863E08C2FD7
:100DC0000E946E0D21C081E00E94890D0230E0F08A
:100DD00082E00E94890D18C0112331F0002391F2A6
:100DE0008D2F0E94470410C0002399F2D93349F493
:100DF0001FEF27EE33E0115020403040E1F700C0F4
:100E000000008D2F0E949D0488EF8C0D843020F40B
:100E10000E94312B0E94DC03DD20C9F00E94DC0C13
:100E200080FD15C0F70112820E94D60C0E944C086A
:100E3000C7010E9448070E94D60CDF91CF911F91F5
:100E40000F91FF90EF90DF90CF900C946D08DF91A1
:100E5000CF911F910F91FF90EF90DF90CF90089569
:100E60000F931F93CF93DF93EC01688179818A817F
:100E70000E948E098C010E94E9080E94DA07B801DD
:100E8000CE010E94FF04DF91CF911F910F91089531
:100E9000CF93DF93EC01988189812B813C81232BB7
:100EA00031F08F3F31F481E09F3F19F403C081E0BE
:100EB00001C080E080FD1DC0CE010E946B03811146
:100EC00010C00E94E00C8823A1F08A81882389F059
:100ED00080914F0582FD0DC082E0DF91CF910C948F
:100EE000890DCE010E943007CE01DF91CF910C9485
:100EF0004C03DF91CF91089580E090E00E94682B31
:100F000080E090E00E947E2B0E94070D0E94290D38
:100F10000E94A1150C94701480911D0290911E02E4
:100F20000E94402C0C947C070E94F70C0C948C07B8
:100F300092959F70963079F010F4925001C09A50BB
:100F4000923068F4803F69F018F4883E40F409C09C
:100F5000843F29F406C0883E20F0813F11F080E0F4
:100F6000089581E00895FC01808191810E948309A8
:100F70000E9498070895CF93DF9300D000D01F926E
:100F8000CDB7DEB70F900F900F900F900F90DF91BD
:100F9000CF910895CF93DF9300D000D000D0CDB78C
:100FA000DEB726960FB6F894DEBF0FBECDBFDF9139
:100FB000CF910895089508950C94DB070C94DC07F5
:100FC0000E94DE0760930003709301038093020385
:100FD000909303030C947C070C94E0070F931F93EA
:100FE000009100031091010320910203309103034B
:100FF000602B712B822B932B1F910F910C94E00788
:101000000F931F930091000310910103209102039D
:101010003091030360237123822393231F910F9147
:101020000C94E0070F931F930091000310910103AC
:1010300020910203309103036027712782279327B1
:101040001F910F910C94E0070C94DB070E94240879
:101050006093FC027093FD028093FE029093FF0266
:101060000C947C0760E070E0CB010C9426080F9391
:101070001F9341E050E060E070E08A019B0104C0F2
:10108000000F111F221F331F8A95D2F7C901B80123
:101090001F910F910C9426080F931F9341E050E08D
:1010A00060E070E004C0440F551F661F771F8A95EB
:1010B000D2F78091FC029091FD02A091FE02B091C6
:1010C000FF028A019B01082B192B2A2B3B2BC901FC
:1010D000B8011F910F910C9426080F931F9341E0C4
:1010E00050E060E070E004C0440F551F661F771F9A
:1010F0008A95D2F740955095609570958091FC0245
:101100009091FD02A091FE02B091FF028A019B0125
:10111000082319232A233B23C901B8011F910F91EA
:101120000C9426080F931F9341E050E060E070E0BC
:1011300004C0440F551F661F771F8A95D2F7809110
:10114000FC029091FD02A091FE02B091FF028A0183
:101150009B01082719272A273B27C901B8011F919E
:101160000F910C9426080F931F930091FC0210918D
:10117000FD022091FE023091FF02602B712B822B29
:10118000932B1F910F910C9426080F931F9300919E
:10119000FC021091FD022091FE023091FF026023BB
:1011A0007123822393231F910F910C9426080F9390
:1011B0001F930091FC021091FD022091FE023091DC
:1011C000FF0260277127822793271F910F910C94AC
:1011D000260808952FE0929F800D1124E82FE695B0
:1011E000E695E695877051E001C0550F8A95EAF7BC
:1011F00085E0E89FF0011124E653FD4F20E030E048
:1012000070E04081CB01022E02C0969587950A942A
:10121000E2F78170819584278523842781932F5F4E
:101220003F4F2530310569F708952FE0929F800DDB
:101230001124682F669566956695982F977085E0BE
:10124000689FB001112440E050E080E0FB01E40F12
:10125000F51FE653FD4F208130E0092E02C0369580
:1012600027950A94E2F721703327042E01C0220F3C
:101270000A94EAF7822B4F5F5F4F4530510531F7F3
:101280000895BF92CF92DF92EF92FF920F931F9338
:10129000CF93DF938C01C090FC02D090FD02E090D0
:1012A000FE02F090FF028091000390910103A09153
:1012B0000203B0910303C82AD92AEA2AFB2ACFE104
:1012C000D0E0D701C6010C2E04C0B695A79597951E
:1012D00087950A94D2F780FD04C0219790F7B12C2E
:1012E00007C0BC2EB8018C2F0E9497100197A9F35C
:1012F0008B2DDF91CF911F910F91FF90EF90DF9099
:10130000CF90BF900895CF93DF93EC010E944109E5
:10131000BE010E949710DF91CF9108951F93CF9344
:10132000DF93EB019091C902992321F0CB010E9438
:10133000830913C0882349F0CB010E944109182F6B
:10134000682FCE010E94EA0804C0CB010E94150953
:10135000182FBE01812F0E949710DF91CF911F910E
:1013600008951F93CF93DF93C091040316E08091FB
:101370000503C81799F0D0E01C9FF0011D9FF00DE8
:101380001124EA5FFC4F4081518162817381848125
:1013900095810E94CA072196C770E9CFDF91CF914E
:1013A0001F9108954091360350913703609138039F
:1013B0007091390380913A0390913B030C94CA07D2
:1013C000EF92FF920F931F93CF93DF9380913B0394
:1013D00082958F7009F065C080913803882309F4E5
:1013E00060C080910403F0900503109136030091D2
:1013F00037036091390370913A0391E01F3F09F080
:1014000090E0C0911B02D0911C02292F96E0E92E9A
:101410008F1509F446C06115710521F00F3F21F0C9
:1014200030E003C031E001C0322F90E030FD36C023
:10143000E89EF001E99EF00D1124DF01AA5FBC4F88
:1014400011963C911197301329C03C91311326C05D
:1014500012963C911297311121C013964D915C91D7
:101460001497461B570B4C175D07C0F480913B0344
:101470008F70806180933B03E55FFC4F80818F70AC
:101480008061808386E393E00E944807DF91CF91DB
:101490001F910F91FF90EF900C94B1090196877006
:1014A000B7CFDF91CF911F910F91FF90EF900895EB
:1014B0009F92AF92BF92CF92DF92EF92FF920F93E3
:1014C0001F93CF93DF93CDB7DEB761970FB6F89434
:1014D000DEBF0FBECDBF8C0185E0F801DE011D9699
:1014E00001900D928A95E1F7D8011296EC909091B7
:1014F0003603E09137032091390330913A032115E7
:10150000310531F0EF3F31F481E09F3F19F403C022
:1015100081E001C080E0B82FB1709B2E80FD47C1F3
:10152000D8014C9111965C9111971396AD90BC9097
:10153000149786E3C82E83E0D82EF0903803B501C7
:10154000621B730B20911B0230911C02FF2009F4D7
:10155000D9C080913B036217730708F095C0282F0C
:10156000207F09F052C05E1313C0491311C0FE2C36
:10157000E1100EC08F70806180933B030E94D209FE
:10158000C6010E94480780913B03F80185834DC145
:10159000AB2831F05F3F31F481E04F3F19F403C0D5
:1015A00081E001C080E080FD03C081E08E2502C0A3
:1015B00080E090E0F82FF170FF2E80FF1CC080913A
:1015C00004032091050336E0821709F40BC190E073
:1015D000389FF001399FF00D1124EA5FFC4F6181C3
:1015E000561306C06081461303C06281E61203C031
:1015F00001968770E9CFFE2CEE2009F416C1809188
:101600003B03816080933B0354C05E1306C04913C3
:1016100004C0E11002C0F80199C0C8010E94B307DC
:10162000882361F1EE2051F120913B03822F8295B6
:101630008F7090E0029774F0809136039091370399
:1016400098878F831986BB86AA862C87CE0107963A
:101650000E94480786E0F801A6E3B3E001900D92EE
:101660008A95E1F70E94E0090E94D2090AC05E173C
:1016700011F1C8010E94B30781112CC0C8010E945A
:101680004807FF24F394D1C0282F207F81F77A2DBB
:10169000B98AA88A6E2D89890E94BB0786E393E0E8
:1016A0000E94480786E0D6011D928A95E9F70E94BC
:1016B000D209F12CBAC04913DCCFE110DACFF8011E
:1016C0008583C8010E94480786E0D6011D928A954D
:1016D000E9F7ABC0EE2091F220913B03822F829577
:1016E0008F7090E002970CF4B5CF80913603909103
:1016F00037039A8389831B82BD82AC822E83CE01FD
:101700000196A6CF6217730708F044C0FE2CEE20A6
:1017100009F4B4CF5E1330C049132EC020913B03AF
:1017200020FD21C0822F82958F70482F50E04115F7
:101730005105C9F0F80125834F30510541F08F5F05
:10174000982F9295907F822F8F70892B8583C80167
:101750000E94480786E0F801A6E3B3E001900D92ED
:101760008A95E1F73CC086E0F801A6E3B3E001907A
:101770000D928A95E1F759C0C8010E94B307811103
:1017800069CF80913B03816080933B03C8010E9435
:1017900048074BC07A2DB98AA88A6E2D89890E9484
:1017A000BB0786E0D6011D928A95E9F718C0EE20A6
:1017B00009F464CFC8010E94B307F82E882309F406
:1017C0005DCF86E0F801A6E3B3E001900D928A9523
:1017D000E1F786E393E00E9441040E94E0090E9441
:1017E000D20923C04D875E878D859E850E9483091F
:1017F000292F22952F70223028F49F7039F0811103
:1018000005C00BC0243028F49F7049F4805E8830F6
:1018100020F0C8010E9448079F2CF92C06C0D8016F
:1018200015969C91907F91F7F8CF8F2D61960FB60A
:10183000F894DEBF0FBECDBFDF91CF911F910F9106
:10184000FF90EF90DF90CF90BF90AF909F90089562
:101850001F93CF93DF93CDB7DEB72C970FB6F894D5
:10186000DEBF0FBECDBF4F83588769877A878B87CE
:101870009C87CE0107960E94580A8823D1F09F8149
:1018800088852A853B85232B31F08F3F31F481E019
:101890009F3F19F403C081E001C080E080FD47C094
:1018A0004F81588569857A858B859C850E94CA07FA
:1018B0003EC086E0FE013796DE01119601900D9242
:1018C0008A95E1F7FF81E8856A857B856115710559
:1018D00031F0EF3F31F481E0FF3F19F403C081E0C4
:1018E00001C080E080FD23C02091050330E0C901E4
:1018F0000196877099274091040350E0841795075B
:10190000F1F1F983EA837D836C8396E0929FD001A5
:10191000939FB00D1124AA5FBC4FFE013196019038
:101920000D929A95E1F7809305030E94B10916E0A4
:101930008091040390910503891771F1189FC001EC
:1019400011248A5F9C4F0E94580A882329F1E09154
:1019500004031E9FF0011124EA5FFC4F4081518176
:1019600062817381848195810E94CA0780910403FA
:1019700090E001968770992780930403D9CF0E9445
:1019800094071092050310920403E6E3F3E086E067
:10199000DF011D928A95E9F72C960FB6F894DEBF09
:1019A0000FBECDBFDF91CF911F91089580915C0351
:1019B000859585958595089580915C038770089538
:1019C00090915C03977081E009F480E00895809124
:1019D0007F03089590917F03892B80937F0308955F
:1019E000809590917F03892380937F0308951092BF
:1019F0007F03089590917E03892B80937E03089541
:101A0000809590917E03892380937E0308951092A0
:101A10007E03089580915D03089508950C940D0D43
:101A20000C940E0D90914F0592FD08C090915D03AE
:101A3000981721F080935D030C94100D0895809108
:101A40005D03882329F010925D0380E00C94100D53
:101A50000895CF93DF93E0911D02F0911E028091D3
:101A60007F038083E0911D02F0911E02908180919E
:101A70007E03892B808380915D03882381F0E09130
:101A80001D02F0911E029081892B808380911D029E
:101A900090911E020E94942B81110E941F0DC091F3
:101AA0001D02D0911E0240E250E06CE373E0CE01D3
:101AB0000E943035892B69F080E2FE01ACE3B3E08F
:101AC00001900D928A95E1F7CE01DF91CF910C94B0
:101AD000402BDF91CF9108950C940D0D90914F05FF
:101AE00092FD10C098E0899F90011124262B20932D
:101AF0005C030E944C0880915C03859585958595D3
:101B00000C946C0D0C944C0810925C0380E00C94C7
:101B10006C0D20915C038095822380935C03982F49
:101B2000977099F430E0482F082E000C550B2417BD
:101B3000350759F090914F0592FD07C08595859521
:101B400085950E946D080C94840D089590914F0521
:101B500092FB222720F9281769F080FB92F99093D5
:101B60004F0580914E0590914F050E94F40D82E043
:101B70000C94890D089580914F0582FB882780F988
:101B800091E089270C94A60D81E00C94A60D80E0CD
:101B90000C94A60D6FEF7FEF80E090E00C949235EF
:101BA00080E090E00E945E3521E0893E9E4F09F082
:101BB00020E0822F089582E090E00C94563583E077
:101BC00090E00C945635CF9384E090E00E94563517
:101BD000C82F82E290E00E9456352C2F30E0A901F8
:101BE000582BCA01CF910895CF93C92F682F84E055
:101BF00090E00E9474356C2F82E290E0CF910C94BB
:101C00007435AB01BC018FE090E00C948635AB01DC
:101C1000BC0183E190E00C94863560E070E0CB017C
:101C20000C94070E60E070E0CB010E94010E0C9452
:101C30000D0E69EE7EEF80E090E00E94923560E04C
:101C400082E090E00E94743560E083E090E00E94C2
:101C50007435109200031092010310920203109247
:101C6000030360E084E090E00E94743560E082E26B
:101C700090E00E94743560E085E090E00E94743549
:101C800060E086E090E00E9474356FEF87E090E0BE
:101C90000E94743540E050E0BA0188E090E00E9474
:101CA000863560E08DE090E00E94743540E050E0C1
:101CB000BA0188E190E00E94863560E087E190E01B
:101CC0000E94743540E050E0BA018CE190E00E943F
:101CD000863560E070E080E290E00E94923540E05E
:101CE00050E0BA0188E190E00E9486350C94120E13
:101CF0000C94190E682F8EE090E00C9474350E94BD
:101D0000FA2C60938E0370938F03809390039093CB
:101D1000910360938A0370938B0380938C03909359
:101D20008D03089585B7806885BF85B7806885BFB6
:101D3000089581E008950C94990E08950C949D0ED9
:101D40000C949D0E0C94A00E0C949D0E0C94A40E5D
:101D50000C949D0E0E94920E83E791E10E94272B26
:101D60000E94A80E0C94A60E0E949E0E0C949D0E2E
:101D70000E948D110E94DB030C94E1230E94E52C4C
:101D80000E9472120E94B80E0C94A20E5F926F9283
:101D90007F928F929F92AF92BF92CF92DF92EF92FB
:101DA000FF920F931F93CF93DF93CDB7DEB72A97A0
:101DB0000FB6F894DEBF0FBECDBF0E948712E82E8B
:101DC00081110E947F0E30E8832E33E0932E00E0D5
:101DD00010E0502E802F0E94B1115C01F40161903F
:101DE00071904F016826792661147104B1F40F5F78
:101DF0001F4F0530110569F78FEF89838A831B8296
:101E00000E94EE2C8160782F9D838C8349815A81BA
:101E10006B818D810E94F70343C08091920381FD05
:101E20000E94BA11F12CCC24C394D12CC3018C2173
:101E30009D21892B71F10E949B0EAC20BD2088232F
:101E4000A1F0FE825F8281E0A114B10409F480E078
:101E500088870E94EE2C8160782F9A8789874E812F
:101E60005F8168858A850E94F703000F111FF801C2
:101E7000E058FC4F80819181C826D926D182C0824A
:101E800041E0AB2809F440E06F2D852D0E94FB1E38
:101E900007C0F394CC0CDD1CFFE0FF12C7CFA7CF27
:101EA00081E0E11001C080E02A960FB6F894DEBF11
:101EB0000FBECDBFDF91CF911F910F91FF90EF909B
:101EC000DF90CF90BF90AF909F908F907F906F905A
:101ED0005F9008950E94C60E0E9418230E948E14DF
:101EE0000C94EC03CF93DF930E949C10EC018115BE
:101EF00021E5920708F045C0811530E5930708F009
:101F000094C0883E910528F5803E910508F0F8C000
:101F1000883A910570F4853A910508F07CC08130CB
:101F2000910509F475C008F4E8C0049708F0E8C00A
:101F3000E4C08F3B910508F0E0C0C85AD0E0CC0F58
:101F4000DD1FC059DD4F0990D881C02DCE019464AA
:101F5000D8C0811540E2940758F4811551E09507E7
:101F600008F0CEC08D3E910508F4C7C09065C9C089
:101F7000C11580E4D80708F4C0C0DF70CE01906AB4
:101F8000C0C0811525E59207A8F4811534E59307B3
:101F900008F095C0811543E5940708F07BC08115D2
:101FA00052E5950708F061C0D82FCC27CE01816F8C
:101FB000906AA7C0C11589E5D807A0F4C11528E526
:101FC000D20708F082C0C11536E5D30708F095C0E6
:101FD0008C2F0E9430118F7190E0D82FCC27CE012A
:101FE00090628FC0C1154AE5D40708F474C0CE01D1
:101FF00090568115904208F080C08D2F8F710E94FD
:102000003011DD27D0628F71AE01582BCA0179C023
:1020100081E090E076C0C55AD0E0C256DD4F88819D
:10202000C82FD0E0CE0190646CC074E0969587957F
:102030007A95E1F7282F23703C2F337081E090E0F0
:1020400002C0880F991F3A95E2F79C68AC01522BA9
:102050009A019C2F9F709695969550E2959FE0016E
:102060001124C9018C2B9D2B4CC08370992721E032
:1020700030E002C0220F331F8A95E2F79C2F96951D
:10208000969580E2989FE0011124C22BD32BCE01BC
:102090009C6837C08370992721E030E002C0220F8E
:1020A000331F8A95E2F79C2F9695969540E2949F70
:1020B000E0011124C22BD32BCE019A6822C0D82F65
:1020C000CC27CE01846F906A1CC0DC2FCC27CE01B8
:1020D000806F906A16C08C2F8F700E94301194E030
:1020E000D695C7959A95E1F7CF70D0E0DC2FCC2735
:1020F000D0699E01282BC90104C080E090E001C096
:10210000CE01DF91CF9108952BE4829FC00111246D
:10211000FC012FE0729FE00DF11D1124E60FF11D6F
:10212000EE0FFF1FE851FE4F8591949108950E9494
:1021300084100E94720F08958238910569F1B0F4FD
:102140008133910509F46DC048F48932910509F491
:1021500063C08A32910509F469C0089585339105F9
:1021600009F455C089339105B9F00895833E91056E
:1021700069F138F4803E9105B1F0823E910509F194
:102180000895863E9105A9F1873E9105B9F1843EF7
:10219000910509F064C023C020914E0520FD4FC079
:1021A00021FD4DC0089580914E0580FD44C0809171
:1021B0004F0580FF44C080914E0584FD42C083EEF0
:1021C0004DC080914E0582FF38C0F5CF80914E05FD
:1021D00082FD33C080914F0580FD31C0ECCF8091EE
:1021E0004F0581FF32C080914E0584FD2AC087EEE5
:1021F00035C080914E0583FF26C0F5CF80914E05F6
:1022000083FD21C080914F0581FD1FC0ECCF8091DF
:102210004E0585FD1CC01DC080914E0585FD19C071
:1022200016C080914E0586FD16C017C080914E05E0
:1022300086FD13C010C089E311C082EE0FC080EE8E
:102240000DC080E00BC086EE09C084EE07C089E2B5
:1022500005C085E303C08AE201C081E390E00895F0
:1022600090914E0592FF0DC0282F2871283019F447
:10227000877F846006C0282F2471243011F48B7F5F
:10228000886093FF0DC0282F2871283119F4877EAC
:10229000846106C0282F2471243111F48B7E88615B
:1022A00020914F0520FF0DC0382F3871383019F4B8
:1022B000877F816006C0382F3171313011F48E7FF5
:1022C000886021FF0DC0282F2871283119F4877EDE
:1022D000816106C0282F2171213111F48E7E886121
:1022E00094FD877E089580E008950C94CA0D0E94A5
:1022F00087128FEB9DE50197F1F700C000000E9467
:10230000871280E00E94B11180FF04C00E94751105
:102310000C94572D08950C9477110E94D00D8111C3
:1023200002C00E94780E0E94DB0D809392030E94EF
:10233000E30D90934F0580934E050E948B110E94F0
:10234000DF0D682F70E080E090E00E94EC07609164
:10235000FC027091FD028091FE029091FF020C94AC
:102360002408E82FF0E0EE0FFF1FE65AFA4F8081B5
:1023700091810895089580EA8A95F1F7089500C043
:1023800008950C94BB1108950C94C3110C94C411BE
:102390000C94C3110C94C811F894E82FE295EF70D7
:1023A000F0E031A1282F2F7081E090E001C0880F6C
:1023B0002A95EAF7982F9095932391A392A1892BC0
:1023C00082A3789408950F931F93CF93DF93C0EB6C
:1023D000D2E089918F3F11F00E94CC1182E0C53B81
:1023E000D807B9F7C1EAD2E000EB12E089918F3F3C
:1023F00011F00E94CC110C171D07C1F7DF91CF918E
:102400001F910F910895BF92CF92DF92EF92FF92AA
:102410000F931F93CF93DF938C01C62FD0E0CE0193
:1024200080559D4F6C01FC0190819F3F09F450C085
:10243000B62EF894E92FE295EF70F0E081A19F703D
:1024400021E030E001C0220F9A95EAF7822B81A3A8
:1024500082A12095282322A378940E94BF11E1EA4B
:10246000F2E040EB52E021E030E0E12CF12C619110
:102470006F3F89F0A62FA295AF70B0E090968C9137
:1024800090E06F7002C0959587956A95E2F780FDA0
:1024900002C0C90102C080E090E0E82AF92A220FB8
:1024A000331F4E175F0719F7F60180818F3F11F038
:1024B0000E94CC1161E0E114F10409F460E08B2D7D
:1024C0000E94C111CC0FDD1FC00FD11FF982E8821D
:1024D000DF91CF911F910F91FF90EF90DF90CF9000
:1024E000BF9008950E94E3118AE0EAE5F5E0DF017C
:1024F000982F1D929A95E9F7E0E5F5E0DF011D922E
:102500008A95E9F785E00E94D2120C945703FF9256
:102510000F931F93CF93DF93CDB7DEB72A970FB6F4
:10252000F894DEBF0FBECDBF8E010F5F1F4F8AE054
:10253000F80111928A95E9F7F12C6F2DC8010E94DC
:102540000312F394F5E0FF12F8CF4AE050E0B8012F
:1025500080E595E00E943035FF24F394009709F45C
:10256000F12C892B41F08AE0F801A0E5B5E001905B
:102570000D928A95E1F72F2D45E06AE575E080E53B
:1025800095E00E94D3120E9459038F2D2A960FB610
:10259000F894DEBF0FBECDBFDF91CF911F910F9199
:1025A000FF9008950895FF920F931F93CF93DF93A9
:1025B000F82E092F162FD72FC42F222349F081E0A0
:1025C000809395030E94EE2C909394038093930341
:1025D000809195038823D9F080919303909194037F
:1025E0000E94062D039798F0EF2DF02FA12FBD2FFD
:1025F00080E090E04C2F50E08417950734F421914F
:1026000031912D933D930196F7CF10929503DF9171
:10261000CF911F910F91FF9008950E94222F0E9449
:10262000BE0E0C942E2F0E94322F0E946A0F0C9423
:102630004C2F0E948C2C0E94092F0E94AA0E0E94EF
:102640000D130E9413130E94B40EFBCF80919C03C4
:1026500080FF06C06091240270E0660F771F26C0DD
:1026600081FF04C06091240284E005C082FF07C09E
:102670006091240288E0689FB001112417C09091F6
:102680009B039923D1F060912302961788F720913C
:10269000240288E0289F90011124929FA001939F1B
:1026A000500D112470E0CA010E9470346038710529
:1026B00040F46115710519F406C068E070E0862FDA
:1026C00008958FE7089581E0089580919C0380FF2D
:1026D00008C06091200270E07595679575956795C3
:1026E00021C081FF06C06091200270E0759567955A
:1026F00019C082FF04C06091200270E010C0909168
:102700009A03992399F060911F029617A0F7809180
:102710002002899FC001112470E00E94703460384B
:10272000710540F46115710519F406C061E070E0AF
:10273000862F08958FE7089581E008958D3E21F456
:102740000E942613819504C08E3E29F40E94261310
:102750008093A00308958F3E21F40E942613819553
:1027600004C0803F29F40E94261380939F0308959C
:10277000893F19F40E94651305C08A3F31F40E9415
:10278000651381958093A10308958B3F21F40E94E6
:102790006513819504C08C3F29F40E9465138093D2
:1027A000A20308959FE0980F983078F421E030E07C
:1027B000A90102C0440F551F9A95E2F7CA019091F2
:1027C0009E03892B80939E0308958D3F21F4809171
:1027D0009C0381600BC08E3F21F480919C0382603A
:1027E00005C08F3F29F480919C03846080939C03F3
:1027F00008958D3E39F49091A00397FF35C0109253
:10280000A00359C08E3E29F49091A0031916BCF381
:102810002BC090919F038F3E29F497FF25C0109203
:102820009F0349C0803F19F41916CCF31DC0909145
:10283000A103893F29F41916BCF41092A1033BC0EF
:102840008A3F19F497FF10C0F8CF8B3F39F490916D
:10285000A20397FF09C01092A2032DC08C3F21F460
:102860009091A2031916BCF39FE0980F983080F462
:1028700021E030E0A90102C0440F551F9A95E2F70C
:10288000CA01809590919E03892380939E0313C073
:102890008D3F21F480919C038E7F0BC08E3F21F4ED
:1028A00080919C038D7F05C08F3F29F480919C030C
:1028B0008B7F80939C0380919F03811106C0809140
:1028C000A003811102C010929B038091A10381118A
:1028D00006C08091A203811102C010929A0308954C
:1028E0000E94EE2C20919F03211104C02091A0038F
:1028F000222321F090939903809398032091A103C0
:10290000211104C02091A203222321F09093970368
:10291000809396038DE993E00C945A2BEF92FF92EB
:102920000F931F93CF93DF9300D000D000D0CDB78B
:10293000DEB786E0EDE9F3E0DE01119601900D923D
:102940008A95E1F7E0909F03F090A0030091A10326
:102950001091A20310929F031092A0031092A10362
:102960001092A203E11003C0FF2009F45DC0809122
:102970009803909199030E94062DAC0190919B03BE
:10298000992339F02091250230E02417350758F0BB
:102990004BC0209126028AE0289F90011124241721
:1029A000350718F041C09F3F19F09F5F90939B033C
:1029B000EE2061F00E9426131E1414F09FEF01C058
:1029C00091E0989F902D112490939F03FF2061F038
:1029D0000E9426131F1414F09FEF01C091E0989FEE
:1029E000902D11249093A00330919F033323E1F0A5
:1029F0002091A0032223C1F045EB3403C001112430
:102A0000992319F090939F0303C081E080939F0363
:102A100035EB2303C0011124992319F09093A003EF
:102A200003C081E08093A003011103C0112309F4C6
:102A30005DC080919603909197030E94062DAC0192
:102A400090919A03992339F02091210230E02417C4
:102A5000350758F04BC0209122028AE0289F900150
:102A600011242417350718F041C09F3F19F09F5FCC
:102A700090939A03002361F00E946513101614F0DE
:102A80009FEF01C091E0989F902D11249093A10396
:102A9000112361F00E946513111614F09FEF01C01D
:102AA00091E0989F902D11249093A2033091A1035F
:102AB0003323E1F02091A2032223C1F045EB34033C
:102AC000C0011124992319F09093A10303C081E060
:102AD0008093A10335EB2303C0011124992319F03E
:102AE0009093A20303C081E08093A20380919F038F
:102AF00081110BC08091A003811107C08091A103B7
:102B0000811103C08091A20381110E947014EB8295
:102B1000FC820D831E8386E0FE013196ADE9B3E0B1
:102B200001900D928A95E1F726960FB6F894DEBFD4
:102B30000FBECDBFDF91CF911F910F91FF90EF900E
:102B40000895EDE9F3E086E0DF011D928A95E9F74B
:102B500010929B0310929A0310929C030895EF9297
:102B6000FF920F931F93CF93DF938B01682F111167
:102B70000AC0442329F0E82FF0E0EC5EFC4F64919A
:102B8000762F862F75C0212F30E0E82FF0E0442308
:102B900021F0EC5EFC4FE491F0E046E0049FC001C0
:102BA0001124CFEFD0E0BE010E945C344BEA460313
:102BB000C001479F900D1124800F911D800F911D22
:102BC000982F990F890FAE01421B530B4E9FD001D6
:102BD0004F9FB00D5E9FB00D11249B2F189FA00139
:102BE0001124452F55278E01041B150B0E9FA001A4
:102BF0000F9F500D1E9F500D11247E01E81AF10801
:102C0000E29E8001E39E100DF29E100D1124212FF3
:102C10003327C21BD30BCE9F9001CF9F300DDE9F79
:102C2000300D112462307105A9F048F46115710569
:102C300069F061307105C9F48B2F752F0DC06430B8
:102C4000710581F058F06630710579F47E2F8B2F75
:102C5000932F0DC0832F7B2F9E2F09C08E2F7B2F8C
:102C6000952F05C08E2F732F02C07E2F852F692FC1
:102C7000DF91CF911F910F91FF90EF90089541E068
:102C80000E94AF15089520E030E0869F212D969F89
:102C9000200D311D1124C9010895BC018230910518
:102CA00008F40895613E8EE1780748F49B0195E0B1
:102CB000369527959A95E1F748E0420F01C04FEF0E
:102CC00091E0242F30E0290F311D35952795229F63
:102CD000F001239FF00DF00D11246E177F0718F4FB
:102CE0004FEF420F04C02F3F39F091E0920F491788
:102CF00040F78FEF890F08958FEF089540912D02CF
:102D000050912E0225E038E0429FC001439F900D74
:102D1000529F900D1124875E994C90932E028093C0
:102D20002D02890F0895482F982F46FD9095E92F81
:102D3000EF739F7046FD9F5FE295EF70EE0FF0E03E
:102D4000EB54FD4F2181299F802D212D1124829547
:102D50008F702295207F822B3081982F930F892F9F
:102D600047FD819580580895E42FF0E0EE0FFF1F96
:102D7000E15BFE4F408134EE439F412D1124E82F4B
:102D8000F0E050E0445E5F4FDA01A21BB1099D0103
:102D9000B7FF03C031952195310993E0220F331F0E
:102DA0009A95E1F7AF01421B530B9A0157FF02C0FE
:102DB00020E030E0582F259F212D1124822F0895E7
:102DC000622F0895E42FF0E0EE0FFF1FE15BFE4F4E
:102DD0006081621B0895E42FF0E0EE0FFF1FE05BBF
:102DE000FE4F6081621B0895A22F50E0FA01EE0FA2
:102DF000FF1FE05BFE4F9081905297FD9195440F2D
:102E0000551FFA01E15BFE4F3081232F30E02A1B72
:102E10003109290F311D97FD3A95620F0895EF9200
:102E20000F931F9393E0099F800111241595079537
:102E30006E2D600F1F910F91EF9008950F93CF9318
:102E4000DF93D72FC82F47FD4195E8E3F0E0CF018E
:102E5000841B910947FD9395889FB001899F700D50
:102E6000700D1124229FC001239F900D900D1124FD
:102E7000860F971F0E944D16682F660F860F682FCA
:102E8000600F7D2F8C2FDF91CF910F9108950F93BD
:102E90001F93522F10E0F801EE0FFF1FE05BFE4F73
:102EA000E081F0E0B0979F015203D001539FB00D35
:102EB0001124000F111FF801E15BFE4F008110E0AB
:102EC0000057110940039001419F300D11242A0F32
:102ED0003B1F37FF02C021583F4F220F232F221FD5
:102EE000330B620F1F910F9108950F931F93522F71
:102EF00010E0F801EE0FFF1FE05BFE4FE081F0E015
:102F0000B097EE0FFF1F9F015203D001539FB00DEA
:102F10001124000F111FF801E15BFE4F008110E04A
:102F200000571109000F111F40039001419F300D00
:102F300011242A0F3B1F37FF02C021583F4F220F99
:102F4000232F221F330B620F1F910F9108950F93B0
:102F50001F9310E0F801EE0FFF1FE15BFE4F908121
:102F6000905797FD9195000F111FF801E05BFE4F00
:102F7000E081F0E0B097DF01AA0FBB1F8D010E0FBB
:102F80001F1F2003D001219FB00D1124E8E3F0E0C2
:102F9000E91BF10997FDF3959F01220F331F89016A
:102FA0000E0F1F1F40039001419F300D11242A0F67
:102FB0003B1F37FF02C021583F4F220F232F221FF4
:102FC000330B620F1F910F9108950F931F93CF93AF
:102FD000DF93D62F072F182FC42F822F0E9493160E
:102FE000EC2FF0E0EE0FFF1FE15BFE4F9081905859
:102FF000890F87FD8195880F682F2CE0629F612DD6
:1030000011246D0F702F812FDF91CF911F910F91A0
:103010000895E42FF0E0EE0FFF1FE15BFE4F90817B
:10302000921B97FD9195292F38E1239F212D112483
:10303000620F08952091680530E1230F08F42FEF07
:1030400060E1822F90E00E944316BC0188EB9BE078
:103050000E945C3480E090E008954095282F429FC4
:10306000412D1124842F089522E8241B08F420E028
:10307000620F0895EF92FF920F939701201B310981
:103080002F3F310519F010F02FEF30E02095382F49
:10309000320F08F43FEF832F0F91FF90EF900895C8
:1030A000FC019B01009721F477FF2BC080E8089575
:1030B000AC0197FF04C044275527481B590BB901A1
:1030C000640F751F37FD0CC0241B350BC901A5E02B
:1030D000880F991FAA95E1F70E94703480E20CC016
:1030E000CB0165E0880F991F6A95E1F7BA01621B71
:1030F000730B0E94703480E6861BF7FF03C0819536
:10310000089580E00895FF920F931F93CF93DF936C
:10311000F62ED72F182FC901C12FC01BBA010E944C
:103120005018982F990F890FC81B2C2F219F212DE4
:103130001124822F6F2D7D2FDF91CF911F910F9141
:10314000FF900895EF920F931F93CF93DF93D62FA5
:10315000C72F182FC9010E19010FBA010E9450186C
:10316000081B202F219F212D1124822F6D2F7C2FB2
:10317000DF91CF911F910F91EF9008950F93CF930F
:10318000DF93D72FC82FC901BA010E945018682FAA
:10319000600F7D2F8C2FDF91CF910F910895EF92CB
:1031A0000F93CF93DF93D72FC82FC9010E19BA0100
:1031B0000E945018602F681B7D2F8C2FDF91CF91BC
:1031C0000F91EF9008950E943F160895E4E6F5E010
:1031D00081E2808380913C0290913D02A0913E0269
:1031E00081839283A3838FE784838FEF858346E077
:1031F00050E06CE170E0CF010E9464351092C6048B
:10320000089580E008950F931F93CF93DF93C82F05
:10321000D62F8A010E9401199FE0C99FF001112455
:10322000EC5FFE4FED0FF11D90819F3F29F0F801FB
:10323000E80FF11D90838F5FDF91CF911F910F9168
:103240000895E091C302F091C4020994E091BF0295
:10325000F091C00209944F925F926F927F928F9289
:103260009F92AF92BF92CF92DF92EF920F931F93F4
:10327000CF93DF932C013B01FC01C081CC0FCC0F1D
:10328000D4E0DC0FD53408F0D4E46091680566958D
:1032900080916A0590916B050E944316182FCD17F7
:1032A00008F044C08C2E912CF401E952FE4F90811D
:1032B000F20181818923C1F1F401EE0FFF1FE15B6F
:1032C000FE4FC080D12CF0E7CF1AD108F401EE0FE9
:1032D000FF1FE05BFE4FA080B12C80E2A81AB1086E
:1032E000CC9C9001CD9C300D300D1124AA9CC001C6
:1032F000AB9C900D900D1124820F931F0E944D16D0
:10330000082F609165057091660580916705E12E33
:103310009501A601F30109950E94E318462F282F75
:10332000672FC4010E942619CF5FB9CF81E0D43442
:1033300008F080E0DF91CF911F910F91EF90DF9027
:10334000CF90BF90AF909F908F907F906F905F9045
:103350004F90089562EA78E10C942B196FE077E1C1
:103360000C942B196FEC78E10C942B19AF92BF924F
:10337000CF92DF92EF92FF920F931F93CF93DF9341
:103380006C015B01FC01C081CC0FCC0FD4E0DC0FE1
:10339000D53408F0D4E460916805669580916A059B
:1033A00090916B050E944316182FCD1778F5EC2EDF
:1033B000F12CF701E952FE4F9081F60181818923BA
:1033C00019F1F701EE0FFF1FE05BFE4F208130E0A7
:1033D00020523109F701EE0FFF1FE15BFE4F4081E4
:1033E00050E04057510960916505709166058091E4
:1033F0006705012FF50109950E94E318462F282F34
:10340000672FC7010E942619CF5FCFCF81E0D43448
:1034100008F080E0DF91CF911F910F91FF90EF9026
:10342000DF90CF90BF90AF90089563E878E10C945F
:10343000B6196EE177E10C94B6196EEB78E10C9455
:10344000B619BF92CF92DF92EF92FF920F931F9324
:10345000CF93DF938C017B01FC01C081CC0FCC0F9B
:10346000D4E0DC0FD53408F0D4E4609168056695AB
:10347000669521E0620F08F46FEF80916A059091E4
:103480006B050E944316B82ECD17F0F4CC2ED12C2C
:10349000F601E952FE4F9081F8018181892391F074
:1034A0006091650570916605809167052B2D4C2F05
:1034B000F70109950E94E318462F282F672FC601B0
:1034C0000E942619CF5FE0CF81E0D43408F080E07D
:1034D000DF91CF911F910F91FF90EF90DF90CF90F0
:1034E000BF90089564EB76E10C94211A60EE76E1CA
:1034F0000C94211A62EE76E10C94211A6BEE76E1BF
:103500000C94211A64EF76E10C94211A65EE77E1B0
:103510000C94211A69E078E10C94211A7F928F9221
:103520009F92AF92BF92CF92DF92EF92FF920F9352
:103530001F93CF93DF936C015B01FC01C081CC0F23
:10354000CC0FD4E0DC0FD53408F0D4E460916805EA
:103550006695669580916A0590916B050E94431669
:10356000182F80E4810F0E94931690E8F92EF80E30
:10357000812F0E94931620E8722E780ECD1700F549
:103580008C2E912CF401E952FE4F9081F60181813D
:103590008923A1F0609165057091660580916705AA
:1035A000E12E0C2F272D4F2DF50109950E94E318D0
:1035B000462F282F672FC4010E942619CF5FDECF28
:1035C00081E0D43408F080E0DF91CF911F910F911A
:1035D000FF90EF90DF90CF90BF90AF909F908F9033
:1035E0007F90089567E477E10C948E1A65E777E1A0
:1035F0000C948E1A67EA77E10C948E1AAF92BF9200
:10360000CF92DF92EF92FF920F931F93CF93DF93AE
:103610008C017B01FC01C081CC0FCC0FD4E0DC0F0E
:10362000D53408F0D4E42091680531E0230F08F484
:103630002FEF30E040E050E06FEF7FEF80E090E070
:103640000E94A6346901CD1708F041C0AC2EB12C00
:10365000F501E952FE4F9081F80181818923A9F19A
:1036600090916E05915097FD15C0292F092E000CE1
:10367000330BF901E259FA4F8189C813F3CF220FB6
:10368000331FF901E259FA4F218D328D2C153D057A
:1036900048F701C096016091680541E0640F08F4A5
:1036A0006FEFC9010E944316AC01609165057091EE
:1036B000660580916705F70109950E94E318462F7A
:1036C000282F672FC5010E942619CF5FBCCF81E04C
:1036D000D43408F080E0DF91CF911F910F91FF90DB
:1036E000EF90DF90CF90BF90AF9008956DE278E1BA
:1036F0000C94FE1A64E378E10C94FE1A2F923F9228
:103700004F925F926F927F928F929F92AF92BF92F1
:10371000CF92DF92EF92FF920F931F93CF93DF939D
:10372000CDB7DEB729970FB6F894DEBF0FBECDBF79
:103730008B834B013A01DB011C91110F110FB4E097
:10374000B10FB983B53410F0E4E4E983F0916E056C
:10375000FA838981181708F07FC0A12EB12CF501DA
:10376000E952FE4F9081D40111968C91892309F47E
:1037700071C020906505309066054B80512CC501C5
:10378000880F991FFC01E15BFE4FFD83EC83C501AF
:10379000880F991F9C01205B3E4F3F832E83FA8147
:1037A0004F1608F047C0E42CF12CAC81BD81BC91D0
:1037B000EB2FF0E0F987E887F701E259FA4F8181B2
:1037C00028853985281B310939872887AE81BF8133
:1037D000CC90D12C8185C81AD108F901EE9F9001B7
:1037E000EF9F300D300D1124CC9CC001CD9C900D6D
:1037F000900D1124820F931F0E944D16082F609187
:10380000680521E0620F08F46FEFF701EE0FFF1F6C
:10381000E259FA4F818D928D0E9443167C019601E8
:1038200048855985B101852DF30109951B01439404
:10383000582EB5CF20916705352D329F312D11249B
:10384000832FB1010E94E318462F282F672FC5014F
:103850000E9426191F5F7DCF81E09981943408F082
:1038600080E029960FB6F894DEBF0FBECDBFDF9182
:10387000CF911F910F91FF90EF90DF90CF90BF906D
:10388000AF909F908F907F906F905F904F903F9000
:103890002F90089520916E0531E0231B08F420E05D
:1038A0004AE358E1BC01822F0C947E1BDF92EF9219
:1038B000FF920F931F93CF93DF938C01DC01CC9188
:1038C000CC0FCC0FD4E0DC0FD53408F0D4E46091F9
:1038D000650570916605809167050E94E318F62ED4
:1038E000E72ED82ECD1798F4EC2FF0E0DF01A95287
:1038F000BE4F8C91D80111969C91982331F02D2DBB
:103900004F2D6E2DCF010E942619CF5FEBCF81E0A6
:10391000D43408F080E0DF91CF911F910F91FF9098
:10392000EF90DF900895AF92BF92CF92DF92EF9227
:10393000FF920F931F93CF93DF938C01FC01C08103
:10394000CC0FCC0FD4E0DC0FD53408F0D4E4E090F9
:103950006605F0906705D09065056D2D7E2D8F2D45
:103960000E94E318C62EB72EA82E609168056D0D33
:103970007E2D8F2D0E94E318F62EE72ED82ECD1720
:10398000B8F48C2F90E0FC01E952FE4F3081F80131
:103990002181232359F030FF04C02D2D4F2D6E2D92
:1039A00003C02A2D4C2D6B2D0E942619CF5FE7CF27
:1039B00081E0D43408F080E0DF91CF911F910F9126
:1039C000FF90EF90DF90CF90BF90AF900895BF929F
:1039D000CF92DF92EF92FF920F931F93CF93DF93DB
:1039E0007C01FC01C081CC0FCC0FD4E0DC0FD534BE
:1039F00008F0D4E4C0906605B09067052091680592
:103A000030E4D32E3D2D329F312D1124D32ECD17EE
:103A100038F50C2F10E0F801E952FE4F9081F701C4
:103A200081818923D9F0F801EE0FFF1FE15BFE4F82
:103A30006081D69EB001112495E0759567959A95A1
:103A4000E1F780916505680F7C2D8B2D0E94E318AE
:103A5000462F282F672FC8010E942619CF5FD7CF86
:103A600081E0D43408F080E0DF91CF911F910F9175
:103A7000FF90EF90DF90CF90BF900895DF92EF928C
:103A8000FF920F931F93CF93DF938C01DC01CC91B6
:103A9000CC0FCC0FD4E0DC0FD53408F0D4E4E090A8
:103AA0006505F0906605D09067056091680566959C
:103AB0006695669580916A0590916B050E94431604
:103AC0000E949316805887FD8195880F282F3D2DE1
:103AD000239F212D1124822FB7010E94E318F62E77
:103AE000E72ED82ECD1798F4EC2FF0E0DF01A95285
:103AF000BE4F8C91D80111969C91982331F02D2DB9
:103B00004F2D6E2DCF010E942619CF5FEBCF81E0A4
:103B1000D43408F080E0DF91CF911F910F91FF9096
:103B2000EF90DF900895DF92EF92FF920F931F9333
:103B3000CF93DF93EC01FC01E952FE4F90816923A2
:103B400081F1D09066050091670510916505E12E21
:103B5000F12C0E941735282FC7018C549F4F68E61F
:103B600071E00E9470348E199F0997FD0396959518
:103B70008795959587952370612F289F600D112457
:103B80007D2D802F0E94E318462F282F672FCE010E
:103B9000DF91CF911F910F91FF90EF90DF900C94E8
:103BA0002619DF91CF911F910F91FF90EF90DF9039
:103BB0000895CF92DF92FF920F931F93CF93DF93DD
:103BC0008C01FC01C281C1111DC06091680520E11A
:103BD000620F08F46FEF80916A0590916B050E9467
:103BE00043166AE070E00E945C34892B49F50E941C
:103BF000173564E470E00E947034F80161810E941E
:103C0000931D1EC0FC01C081CC0FCC0F94E0F92E97
:103C1000FC0EF4E4FF1510F484E4F82ED0E0CF2C71
:103C2000D12CCC15DD053CF4F8016181CE010E9458
:103C3000931D2196F6CFC1E0F3E4FF1508F4C0E030
:103C40008C2FDF91CF911F910F91FF90DF90CF903C
:103C500008951F93CF93DF93FC01E952FE4F20811B
:103C60006223D1F0EC010E941735182F0E941735FE
:103C70008F77782F20E8720F08F47FEF612F809103
:103C800067050E94E318462F282F672FCE01DF918A
:103C9000CF911F910C942619DF91CF911F91089518
:103CA000CF92DF92FF920F931F93CF93DF938C01FC
:103CB000FC01C281C1111DC06091680520E1620F45
:103CC00008F46FEF80916A0590916B050E9443168E
:103CD00065E070E00E945C34892B49F50E9417353D
:103CE00064E470E00E947034F80161810E94291E32
:103CF0001EC0FC01C081CC0FCC0F94E0F92EFC0E4D
:103D0000F4E4FF1510F484E4F82ED0E0CF2CD12C8D
:103D1000CC15DD053CF4F8016181CE010E94291E1D
:103D20002196F6CFC1E0F3E4FF1508F4C0E08C2F34
:103D3000DF91CF911F910F91FF90DF90CF90089569
:103D4000DF92EF92FF920F931F93CF93DF938C013B
:103D5000DC01CC91CC0FCC0FD4E0DC0FD53408F0D3
:103D6000D4E4E0906605F0906705D0906505609119
:103D7000680566956695669580916A0590916B05D4
:103D80000E9443160E949316805887FD8195880FE4
:103D9000682F2CE0629F612D11246D0D7E2D8F2DDB
:103DA0000E943F16F62EE72ED82ECD1798F4EC2F52
:103DB000F0E0DF01A952BE4F8C91D80111969C9181
:103DC000982331F02D2D4F2D6E2DCF010E942619F5
:103DD000CF5FEBCF81E0D43408F080E0DF91CF916A
:103DE0001F910F91FF90EF90DF900895E091C10235
:103DF000F091C2020994CF92DF92FF920F931F932A
:103E0000CF93DF93CDB7DEB728970FB6F894DEBF18
:103E10000FBECDBF182F062FF42E0E94990E8823B7
:103E200009F46FC0FF2049F0AE014F5F5F4F602F74
:103E3000812F0E940319F82E01C0F12C0F2D10E0E4
:103E40008091C7049801280F311D293031056CF18C
:103E500088E090E06C01C01AD10AB80168537B4F2A
:103E6000A60188EC94E00E943D35B80160537B4F79
:103E7000A60180ED94E00E943D35A601440F551F38
:103E8000B801660F771F60527B4F80EE94E00E946E
:103E90003D35B80168527B4FA60188ED94E00E9441
:103EA0003D3588E08F198093C7041091C704DE0167
:103EB000119640E0842F810FF41609F190E05D9196
:103EC000252F30E0BC0169537B4FF901EE0FFF1F36
:103ED000E15BFE4F0081FB010183220F331FF901DB
:103EE000E05BFE4F2081FB012187518B880F991FDA
:103EF000FC01E953FB4F128E118E4F5FDBCF809395
:103F0000C70428960FB6F894DEBF0FBECDBFDF9171
:103F1000CF911F910F91FF90DF90CF9008958091E6
:103F20006A0590916B05A0916C05B0916D0588278D
:103F30009C70AA27BB272AE0B695A79597958795E9
:103F40002A95D1F782309105A105B10571F0833032
:103F50009105A105B10569F040E00197A105B10502
:103F600011F060E008C064E102C044E160E080E07C
:103F700003C044E164E184E10C94F61E5F926F9209
:103F80007F928F929F92AF92BF92CF92DF92EF92E9
:103F9000FF920F931F93CF93DF93D82F80912B0223
:103FA0008D130DC020916405237030E040912C02E8
:103FB00050E081E02417350719F480E001C081E06A
:103FC000817080932A028091690590912902981747
:103FD00039F08093290240E060E080E00E94F61E04
:103FE000DF3009F04CC088E292E00E94B2190AC0AA
:103FF000D43008F08AC0D13009F056C088E292E08F
:104000000E94561CC82F27C00E947E167801EE0C15
:10401000FF1C81FF97C10E0D1F1DF801EE50FC4FD4
:104020001082118212820E941A1800916A05109162
:104030006B0520916C0530916D05DC01CB01800F83
:10404000911FA21FB31F8093BE049093BF04A0933F
:10405000C004B093C104809128028F5F809328022E
:10406000C111B6C282E08093270280912A02811199
:10407000AFC2D111ADC283E080932702A9C2D03173
:1040800008F085C0D73029F488E292E00E94AA198E
:10409000B9CFD83008F04CC0D33009F0A9CF88E2AE
:1040A00092E00E94E71CAECFD23050F480912A02F9
:1040B000882349F140E060E080E00E94F61E23C0C2
:1040C00088E292E00E94931C9DCFDC3108F066C22A
:1040D00080916A0590916B05A0916C05B0916D057A
:1040E000D93109F494C008F09BC14091C2045091A9
:1040F000C3046091C4047091C50484179507A60792
:10410000B70708F038C1C0E0A6CFD53029F488E25F
:1041100092E00E94721A76CFD63028F488E292E0BC
:104120000E943E1D6FCF88E292E00E94151A6ACF6E
:10413000DB3029F488E292E00E94821A63CFDC30FF
:1041400098F4D93029F488E292E00E947A1A5ACF82
:10415000DA3028F488E292E00E94761A53CF88E29F
:1041600092E00E947E1A4ECFDD3029F488E292E080
:104170000E94191A47CFDE3028F488E292E00E94AC
:10418000AE1940CF88E292E00E941D1A3BCFD73192
:1041900029F488E292E00E948A1A34CFD83178F567
:1041A000D33129F488E292E00E94D91D2BCFD4317B
:1041B00098F4D13129F488E292E00E94F61A22CFD5
:1041C000D23128F488E292E00E94F21A1BCF88E2F2
:1041D00092E00E94FA1A16CFD53129F488E292E0D3
:1041E0000E94A01E0FCFD63128F488E292E00E94F0
:1041F000501E08CF88E292E00E94861A03CFDB317E
:1042000009F063CF88E292E00E94761BFBCE4091DA
:10421000BE045091BF046091C0047091C104841722
:104220009507A607B70708F46ECF80912A0281117F
:104230000BC0C0912802CC0FCC0F04E00C0F05344A
:1042400008F454C004E452C040E060E080E00E9402
:10425000F61EC2EFEC2EC3E0FC2E00E010E0CFE72C
:104260000E947E1681FF05C0F70110821182128222
:104270001DC00E947E16B82E0E947E168695782F4D
:104280002C2F720F08F47FEFC801880F991F800F41
:10429000911FFC01EE50FC4F6F016B2D8091670563
:1042A0000E943F16F6016083718382830F5F1F4F68
:1042B000F3E0EF0EF11C0434110591F6BACF8C2F08
:1042C00090E0FC01E952FE4F308120912902232326
:1042D00061F0FC01EE0FFF1FE80FF91FEE50FC4FDD
:1042E0002281408161810E942619CF5FC01738F377
:1042F000C1E0043408F0C0E0043408F4ACCE20E09F
:1043000010E001501109822F90E0801791070CF006
:104310007BCEAC01440F551F480F591F4E505C4FC8
:104320000196FC01EE0FFF1F8E0F9F1FFC01EE5048
:10433000FC4F80819181A281FA0180839183A283C5
:104340002F5FE1CF0E947E16D82E0E947E168695A2
:10435000782F2FE7720F08F47FEF0E0D1F1D0E5000
:104360001C4F6D2D809167050E943F16F8016083F8
:104370007183828358CE0E947E16C82F0E947E16BB
:1043800094E4891BF0F7890F082F10E0F801E95237
:10439000FE4F909129028081892309F4FDC0C1FF5D
:1043A00004C020E040E060E013C00E947E16C82FE9
:1043B0000E947E168695782F2FE7720F08F47FEF04
:1043C0006C2F809167050E94E318462F282F672FD6
:1043D000C8010E9426192091680530E1230F08F4D6
:1043E0002FEF60E1822F90E00E944316BC0184EF22
:1043F00091E00E945C3480916A0590916B05A091D8
:104400006C05B0916D05860F971FA11DB11D80939E
:10441000C2049093C304A093C404B093C50473CEA4
:104420004091EE035091EF036091F0037091F1031E
:1044300084179507A607B70708F465CE80912A026E
:10444000882329F040E060E080E00E94F61E609141
:10445000650570916605809167050E94E318C62F77
:10446000772E682E93EAE92E93E0F92E04E011E00E
:104470002FE4A22E21E0B22E4701C12CD12CF40151
:104480008081F801EC0DFD1D882329F08081262D07
:104490004C2F672D04C0808120E040E060E090E078
:1044A0000E942619F401818181934F01FFEFCF1AF9
:1044B000DF0A26E0C216D10411F7480167018EE039
:1044C000582EF6018685F401882329F08685262D4D
:1044D0004C2F672D04C0868520E040E060E090E02E
:1044E0000E942619F601858586875A94F1E0CF1A35
:1044F000D10821E0821A910837E05312E2CFF70188
:104500008781F801882329F08781262D4C2F672D7C
:1045100004C0878120E040E060E090E00E9426191E
:10452000F7018681F801882329F08681262D4C2FFA
:10453000672D04C0868120E040E060E090E00E94AA
:1045400026190E947E16837091E009F090E0F70131
:1045500096839783FFE0EF0EF11C015F1F4FA016BB
:10456000B10609F089CF0E941A1800916A051091CE
:104570006B0520916C0530916D05DC01CB01800F3E
:10458000911FA21FB31F8093EE039093EF03A0939C
:10459000F003B093F103B7CDC1E05DCDDD3129F477
:1045A00088E292E00E944A1C2DCDDD3128F488E299
:1045B00092E00E947A1B26CDDF3F21F40E948F1FDC
:1045C00082E05ACD809128028F5F809328024ACDE5
:1045D000DF91CF911F910F91FF90EF90DF90CF90DF
:1045E000BF90AF909F908F907F906F905F90089555
:1045F00008950C94F8220E94F9220C94F90208956F
:104600000C94FF22CF93DF93FC01C081CC0FCC0F21
:10461000C450D4E0DC0FD53408F0D4E46D2F8C2FD7
:104620000E9400236D2F8C2FDF91CF910C94FF22DD
:104630004F925F926F927F928F929F92AF92BF92B2
:10464000CF92DF92EF92FF92CF936091F00470913E
:10465000F1048091F2049091F3040E94152D6B01F6
:104660007C010E94FA2C4B015C016093F004709372
:10467000F1048093F2049093F304A091C704E7EC53
:10468000F4E08A2F90E04FEF5FEF60E070E04C19AC
:104690005D096E097F09A91799F0218D328D2901D5
:1046A000612C712C441555056605770510F4815071
:1046B00004C02C0D3D1D328F218F9F5F3296EBCFB2
:1046C0008093C7048091F404811108C0C0916405EF
:1046D0008C2F837019F0C695C69501C0C0E08091FB
:1046E00027028130D9F028F0823089F18330E1F15E
:1046F0005AC01092280280926A0590926B05A0928F
:104700006C05B0926D0589E2E7ECF4E0AEE6B5E049
:1047100001900D928A95E1F781E023C08C2F0E94D1
:10472000BE1FCC2309F43FC00E94FB2288E292E026
:10473000CF91FF90EF90DF90CF90BF90AF909F9080
:104740008F907F906F905F904F900C940223C09356
:104750002B0280916405837080932C020E942119A2
:1047600083E0809327021FC08091C604882351F004
:1047700046E050E06CE170E084E695E00E9464352C
:104780001092C60460916A0570916B0580916C056A
:1047900090916D050E94152D6A3171058105910575
:1047A00010F010922702CF91FF90EF90DF90CF9002
:1047B000BF90AF909F908F907F906F905F904F9041
:1047C0000895E091BD02F091BE02099510926E0528
:1047D000E7E8F5E08FEF9FEF8193919325E0E739CC
:1047E000F207D1F71092C704E0EEF4E08FEF9FEFED
:1047F0008193919324E0E03FF207D1F70E94D00D1E
:10480000811104C00E94780E0E94E61846E050E034
:104810006CE170E084E695E00E9446351092C60493
:10482000809164058C7F11F40C94E6180895CF9361
:10483000C82F882391F08091F40481110EC00E944A
:10484000BE1F10922B0280916405837080932C020E
:104850000E94211983E080932702C093F404CF9132
:104860000895E4E6F5E0208191E09227908310928C
:1048700027029091C604892B8093C604089581E095
:104880000C943124909164059370A1F0811102C0C1
:10489000946007C08E3110F0946703C0880F880FB2
:1048A000982B90936405109227028091C604682B80
:1048B0006093C604089561E00C944224682F90919F
:1048C0006405969596959F5F9E3110F4892F01C0DF
:1048D00081E00C94422481E00C945E24682F909136
:1048E000640596959695915011F0892F01C08DE140
:1048F0000C94422481E00C946E2490916405937092
:1049000071F08093650560936605493C08F048ECBA
:10491000409367058091C604282B2093C604089510
:10492000A4E6B5E01196EC911197F0E0282F1396CC
:104930004C91139712966C91CF0108960C947D249C
:1049400081E00C949024A4E6B5E01196EC911197C7
:10495000F0E0282F13964C91139712966C91CF018B
:1049600008970C947D2481E00C94A324E4E6F5E000
:10497000628120E1620F08F46FEF9181282F43815B
:10498000892F90E00C947D2481E00C94B624E4E619
:10499000F5E0628120E1621B08F460E09181282F3C
:1049A0004381892F90E00C947D2481E00C94C724EE
:1049B000E4E6F5E0438120E1420F08F44FEF9181F6
:1049C000282F6281892F90E00C947D2481E00C9443
:1049D000D824E4E6F5E0438120E1421B08F440E0FE
:1049E0009181282F6281892F90E00C947D2481E0B1
:1049F0000C94E924809368058091C604682B609329
:104A0000C60408952091680530E1230F08F42FEFC4
:104A1000682F822F0C94FA2481E00C9402252091B7
:104A2000680530E1231B08F420E0682F822F0C94E6
:104A3000FA2481E00C940F2560E084E70E941E2791
:104A400061E087E70C941E27CF930E94492A84E7F0
:104A50000E94712587E70E947125C0E021E041E0B6
:104A600061E08C2F0E942226CF5FC434B9F760E04A
:104A700084E70E94362761E087E7CF910C943627C0
:104A8000E7EBF6E06083418324E630E042E050E06B
:104A9000BF01880F0C94002B0F931F93CF93DF93CC
:104AA000082F000FEB0114E21093B706E8EBF6E0D5
:104AB000DE018D91819386E0E83CF807D1F724E68A
:104AC00030E041E150E067EB76E0802F0E94002B60
:104AD000105F6096143B41F7DF91CF911F910F91CA
:104AE0000895CF93DF93C82F4BE06DEF0E944025D0
:104AF00040E06AE08C2F0E9440258FE39CE90197FB
:104B0000F1F700C0000040E060E08C2F0E944025DB
:104B100040E061E08C2F0E94402540E066E08C2F51
:104B20000E94402540E06DEF8C2F0E944025D0E090
:104B300040E06D2F8C2F0E944025DF5FD231C1F7FE
:104B400040E06D2F8C2F0E944025DF5FD432C1F7EB
:104B500040E06D2F8C2F0E944025DF5FD43BC1F7D2
:104B60004BE06DEF8C2F0E94402541E06AE08C2FD6
:104B70000E94402540E06DEF8C2FDF91CF910C9487
:104B80004025FF920F931F93CF93DF9300D000D067
:104B9000CDB7DEB78434910588F5122F042FF62E99
:104BA000BC01660F771F660F771F68527F4F44E086
:104BB00050E0CE0101960E942735898183704A8199
:104BC000282F30E050E9859FC001112489569A4F63
:104BD000FC01E40FF11DB497F0824B81FC01E40F5E
:104BE000F11DB49700834C81840F911DFC01B49793
:104BF0001083F901E55EFA4F81E080830F900F90FA
:104C00000F900F90DF91CF911F910F91FF9008951A
:104C1000FF920F931F93CF93DF93182F062FF42E3D
:104C2000C0E0D0E02F2D402F612FCE010E94C12582
:104C30002196C434D105B1F7DF91CF911F910F9127
:104C4000FF9008955F926F927F928F929F92AF92A2
:104C5000BF92CF92DF92EF92FF920F931F93CF9369
:104C6000DF9300D000D0CDB7DEB7862E942E522E23
:104C700024E0829FC0011124BC0168527F4F44E0B0
:104C800050E0CE0101960E9427352A8130E0C9010B
:104C90008497FC0197FD379673E0F595E7957A9533
:104CA000E1F74B8150E08A0104521109980117FF86
:104CB00002C0295F3F4F63E0359527956A95E1F77C
:104CC0004C8150E05A0164E2A61AB1083501B7FEE2
:104CD00004C03A017DE1671A710843E07594679456
:104CE0004A95E1F758E0C52ED12CB6010E947034E8
:104CF0007C01C801B6010E9470348C01C501B60167
:104D00000E947034FF274981FF24542F537088205C
:104D100081F062E1569FE00DF11D1124E950FB4F37
:104D200061E070E001C0660FEA94EAF75081652BFC
:104D300010C072E1579FE00DF11D1124E950FB4FA7
:104D400061E070E001C0660FEA94EAF76095508177
:104D50006523608333271127542F5370992089F0DE
:104D600062E1569F200D311D1124F901E950FB4FDE
:104D700021E030E001C0220F0A95EAF73081232BB1
:104D800011C072E1579F200D311D1124F901E95026
:104D9000FB4F21E030E001C0220F0A95EAF7209591
:104DA00030812323208377249927942F93709301B4
:104DB0005520A1F052E1959F200D311D1124F901DC
:104DC000E950FB4F21E030E0B90102C0660F771FC8
:104DD0008A95E2F7CB019081892B14C072E1979FED
:104DE000200D311D1124F901E950FB4F21E030E085
:104DF000B90102C0660F771F8A95E2F7CB01809553
:104E00009081892380834370E42FF0E0EB50FB4FC7
:104E100081E080830F900F900F900F90DF91CF91E2
:104E20001F910F91FF90EF90DF90CF90BF90AF90C8
:104E30009F908F907F906F905F900895CF93DF93B6
:104E4000262F30E0E901C55EDA4F9881992351F0B1
:104E500090E9929FB001939F700D112469567A4F8B
:104E60000E944C251882DF91CF910895DF92EF9236
:104E7000FF920F931F93CF93DF93262F30E0A9016A
:104E80004B505B4F7A01FA01908191110AC0F701F2
:104E90001082DF91CF911F910F91FF90EF90DF90E3
:104EA0000895D82EF2E16F9FE001112400E010E098
:104EB000F801EC0FFD1FE950FB4F4081602F8D2D55
:104EC0000E9440250F5F1F4F0231110589F7DFCF88
:104ED000882311F0FA0101C0FB0109941F93CF93BD
:104EE000DF93FB011281111191C0EC010E94E70CCC
:104EF0008272CB3CFCE5DF0709F472C010F5C63CBA
:104F0000ECE5DE0709F453C058F4C43C9CE5D9072E
:104F100009F441C008F044C0C33CDC45C9F136C0C7
:104F2000C83C9CE5D90709F44CC008F445C0C93C0D
:104F3000FCE5DF0709F44AC0CA3CDC4509F44BC074
:104F400025C0C03DECE5DE0709F45DC088F4CD3C2A
:104F50009CE5D90709F44EC008F447C0CE3CFCE5F7
:104F6000DF0709F44CC0CF3CDC4509F44AC00EC051
:104F7000C73D9CE5D90730F4C23DDC4508F046C08A
:104F80008EE042C0CE35DD4509F440C011E03EC0A0
:104F90000E943F243BC04AE754E26BE674E204C03F
:104FA0004BE654E26AE774E20E9468272FC043EBA5
:104FB00054E260EA74E2F8CF40EA54E263EB74E250
:104FC000F3CF45ED54E264EC74E2EECF44EC54E2EE
:104FD00065ED74E2E9CF47EF54E266EE74E2E4CFA8
:104FE00046EE54E267EF74E2DFCF49E155E26CE050
:104FF00075E2DACF4CE055E269E175E2D5CF81E0A8
:1050000003C084E001C089E00E945B24812FDF910E
:10501000CF911F910895CF93DF93EC01FB01828123
:10502000882309F43CC1C430FDE5DF0760F4CB3FC1
:105030009CE5D90788F49E0122503C452431310576
:1050400008F02EC109C0C236EDE5DE0729F0C63AE8
:10505000FDE5DF0709F024C10E94E30D90934F05A1
:1050600080934E05C1318CE5D80709F4C6C008F01D
:1050700042C0C930ECE5DE0709F49BC000F5C5303D
:105080008CE5D80709F485C078F4C330ECE5DE0779
:1050900009F478C008F07AC0C230DC4509F0F5C0E8
:1050A00080914E058160EFC0C7309CE5D90709F4B7
:1050B00078C008F07AC080914E058061E4C0CD30A0
:1050C000FCE5DF0709F487C058F4CB309CE5D9072D
:1050D00009F479C008F07BC080914E0588606FC0EC
:1050E000CF30FCE5DF0709F480C008F082C0809172
:1050F0004E05877FC8C0CE3F9CE5D90709F471C033
:1051000000F5C531FCE5DF0709F485C068F4C3315B
:105110009CE5D90709F475C008F095C00E94940772
:1051200080914E058F77AFC0CC3FFCE5DF07A9F13A
:1051300008F054C0CB3FDC4509F0A7C080914F0573
:1051400040C0C230EDE5DE0709F489C058F4C1154E
:105150008DE5D80709F45AC008F069C080914F0561
:1051600082602FC0C236EDE5DE0709F47CC0C63A86
:10517000FDE5DF0709F481C0C330DD4509F085C0D6
:1051800080E06EC080914E0582607DC080914E05AA
:1051900016C080914E05886076C080914F05826070
:1051A0004FC080914E0580626EC080914E05806434
:1051B0006AC00E94940780914E05806864C0846034
:1051C00062C081603DC080914E058E7F5CC0809141
:1051D0004E058D7F58C080914E0516C080914F05B9
:1051E00018C080914F058D7F2BC080914E058F7E1A
:1051F0004AC080914E058F7D46C080914E058F7BC1
:1052000042C080914E05877F8B7F3DC080914F05C6
:105210008D7F8E7F15C080914E0582FB222720F95D
:1052200091E0922790FB82F990FB83F92CC080914A
:105230004F05982F909591708E7F892B90FB81F967
:1052400080934F0522C00E94940780914E0587FBF2
:10525000222720F991E0922790FB87F914C081E082
:105260000E947A0E12C080914E0584FB222720F9FD
:1052700091E0922790FB84F906C080914E05982F0B
:10528000909590FB80F980934E0580914E0590910A
:105290004F050E94F40D0E94940780E001C081E058
:1052A000DF91CF910895CF93DF9386319C4541F5EF
:1052B000EB010E94E70C982F8A8120911D0230910A
:1052C0001E02882379F09A7A81E009F480E08093C5
:1052D0001D05911102C069E201C065E3C9010E9488
:1052E0002A2C0AC080911D05811102C069E201C00B
:1052F00065E3C9010E94352C0E94290D80E001C0A0
:1053000081E0DF91CF9108950F931F93CF93DF93A7
:10531000C42FD22FFC0182818823C9F0409320053D
:105320000E94EE2C90931F0580931E0580E28C0F47
:10533000883008F057C0C77081E001C0880FCA9557
:10534000EAF7DF91CF911F910F910C94F1048091B6
:105350002005481330C080911E0590911F050E94C2
:10536000062D883C910538F510E21D0FCD17B9F0D8
:1053700080E28C0F883040F4C77081E001C0880F54
:10538000CA95EAF70E94F804183028F581E09D2FAD
:10539000977001C0880F9A95EAF70E94F104802F58
:1053A0000E94E8041830F0F4D77081E001C0880F43
:1053B000DA95EAF70AC080E28C0F883098F4C7705B
:1053C00081E001C0880FCA95EAF7DF91CF911F9164
:1053D0000F910C94F804802FDF91CF911F910F91C2
:1053E0000C94E804DF91CF911F910F9108950F93D2
:1053F0009C01CB01243F4CE5340731F188F4293D71
:10540000FCE53F07D9F02A3D4CE5340779F1283D0A
:105410003C45A9F506E221EE41EE68ED7CE52BC0A6
:10542000263FFCE53F07E1F0A8F0273F3C4539F572
:1054300007E225EE46EE67EF7CE51DC007E225EEAC
:1054400045EE69ED7CE517C006E221EE40EE64EF23
:105450007CE511C007E225EE44EE65EF7CE50BC06C
:1054600006E221EE42EE66EF7CE505C008E221E0AF
:1054700045EE6AED7CE50E94842980E008C0FC01CD
:105480008281882319F01092200501C081E00F91DC
:1054900008951092B9008CE08093B80008959F920F
:1054A000AF92BF92CF92DF92EF92FF920F931F9332
:1054B000CF93DF93B82EEB010E94EE2C6C01C43128
:1054C000D10558F0CF3F8FEFD80759F0CE0164E1F6
:1054D00070E00E945C347B0107C0EE24E394F12C61
:1054E00003C025E0E22EF12C84E8A82E94EA992E40
:1054F0001092BC009092BC000E94EE2C8C01809116
:10550000BC0087FD08C00E94EE2C801B910B8E15FD
:105510009F05A8F32AC08091B900887F883041F0A8
:105520008091B900887F803119F00FEF1FEF1FC005
:10553000B092BB00A092BC000E94EE2C8C01809126
:10554000BC0087FD08C00E94EE2C801B910B8E15BD
:105550009F05A8F30AC08091B900887F883111F0B7
:10556000803419F700E010E00EC00EEF1FEFCF3FC0
:105570008FEFD80709F4BCCFC6010E94062D8C1707
:105580009D0708F4B5CFC801DF91CF911F910F910E
:10559000FF90EF90DF90CF90BF90AF909F900895D5
:1055A0000F931F93CF93DF93EB018093BB0084E8AD
:1055B0008093BC000E94EE2C8C018091BC0087FD82
:1055C0000EC0CF3F8FEFD807C1F30E94EE2C801B97
:1055D000910B8C179D0788F38EEF9FEF0CC02091E5
:1055E000B900287F81E090E0283211F480E090E05B
:1055F000919581959109DF91CF911F910F91089518
:10560000CF92DF92EF92FF920F931F93CF93DF938E
:105610006B018A017901B9010E944F2AE6010C0D44
:105620001D1DC017D10761F424E92093BC00DF9150
:10563000CF911F910F91FF90EF90DF90CF90089541
:1056400097FDF2CFB70189910E94D02AEACF9093BB
:10565000C7028093C602089590932605809325057E
:105660000895E0912505F0912605309721F00190ED
:10567000F081E02D099480E008950E94312B089577
:10568000E0912505F0912605309799F020913B0295
:10569000222359F020914E0527FF07C0DC012C91F1
:1056A00011962C93119726E02C930280F381E02D24
:1056B00009940895E0912505F0912605309739F079
:1056C00022E0DC012C930480F581E02D09940895FB
:1056D00020912305309124052817390771F0909304
:1056E000240580932305E0912505F0912605309748
:1056F00021F00680F781E02D09940895209121057D
:10570000309122052817390771F090932205809374
:105710002105E0912505F0912605309721F00084C0
:10572000F185E02D09940895FC01329680913B02A9
:10573000882331F080914E0587FF02C09EE101C0B1
:1057400096E080E0915028F021912223D9F38F5FD9
:10575000F9CF0895662351F120913B022223E9F00D
:1057600020914E0527FF19C0462F46954695469530
:105770004E31E0F4677021E030E002C0220F331FA9
:105780006A95E2F7FC01E40FF11D828190E0282385
:10579000392381E0232B69F409C0FC013296089675
:1057A0002191621729F0E817F907D1F780E00895F1
:1057B00081E008959C01FC0132969FEF80E04191C9
:1057C000461789F09F3F19F4411101C0982F8F5F50
:1057D0008630A9F79F3F39F0F901E90FF11D97FDD8
:1057E000FA956283089508959C012A5F3F4FFC015A
:1057F0004281461301C01282019682179307B9F7BE
:105800000895262F2695269526952E3168F4FC01BD
:10581000E20FF11D677021E030E001C0220F6A95B0
:10582000EAF78281282B22830895262F2695269534
:1058300026952E3170F4FC01E20FF11D677021E016
:1058400030E001C0220F6A95EAF720958281282373
:105850002283089520913B02222329F020914E05B6
:1058600027FD0C94012C0C94DA2B20913B0222236F
:1058700029F020914E0527FD0C94152C0C94F42B47
:1058800020913B02FC013296222331F080914E059B
:1058900087FF02C08EE101C086E0DF011D928A957C
:1058A000E9F7089508950C94522C83E0809327051E
:1058B0000C94532C811102C081E001C082E08093DE
:1058C00027050C94532C0C945A2C81E080932705C7
:1058D0000C94532C0C94652C08950C946C2C0C9403
:1058E0006D2C0C946C2C0C946C2C0C946C2CCF9315
:1058F0000E94732C0E9487120E94712CC0E08C2F92
:105900000E94B111892B29F4CF5FC530C1F780E027
:1059100001C081E0CF91089508951F920F920FB6B4
:105920000F9211248F939F93AF93BF93809128057B
:10593000811113C08091CB069091CC06A091CD0629
:10594000B091CE064196A11DB11D8093CB069093D8
:10595000CC06A093CD06B093CE06BF91AF919F9198
:105960008F910F900FBE0F901F9018958091D306C6
:10597000843031F10E94C4031092280520E488E1AC
:1059800090E00FB6F894A895809360000FBE209326
:10599000600083B7817F846083BF83B7816083BFEA
:1059A0007894889583B78E7F83BF0FB6F894A895B7
:1059B00080916000886180936000109260000FBE4B
:1059C00008950E9494070C94CD0382E084BD93E077
:1059D00095BD9AEF97BD80936E0008952FB7F89408
:1059E0008091CB069091CC06A091CD06B091CE06C9
:1059F0002FBF08952FB7F8946091CB067091CC0615
:105A00008091CD069091CE062FBF08959C014FB78F
:105A1000F8948091CB069091CC06A091CD06B091E0
:105A2000CE064FBF821B930B0895CF92DF92EF9269
:105A3000FF922FB7F894C090CB06D090CC06E090A0
:105A4000CD06F090CE062FBFA7019601261B370B7F
:105A5000480B590BCA01B901FF90EF90DF90CF902E
:105A6000089578941F920F920FB60F9211248F937E
:105A70009F93AF93BF938091CB069091CC06A0915A
:105A8000CD06B091CE060196A11DB11D8093CB0627
:105A90009093CC06A093CD06B093CE06BF91AF9164
:105AA0009F918F910F900FBE0F901F90189581E0DE
:105AB0008093E00080E28093D8001092C9008FE1CB
:105AC0009EE40197F1F700C0000087E090EBDC0155
:105AD0008093DC069093DD06A093DE06B093DF068C
:105AE0009CE088E10FB6F894A895809360000FBE03
:105AF00090936000FFCF80914C050895089522E0B7
:105B00002093E9002FEF3091E800215035FD06C0C9
:105B100035ED3A95F1F700002111F5CF2091E8001D
:105B200025FF0BC040E050E066E070E00E94BE2F11
:105B30008091E8008E778093E8000895CF93DF93FB
:105B400020913B02222339F020914E0527FF03C00C
:105B500060E222E002C068E021E02093E9002FEF3C
:105B60003091E800215035FD06C035ED3A95F1F74A
:105B700000002111F5CF2091E80025FF1DC0EC01A8
:105B800080913B02811105C040E050E068E070E088
:105B900003C070E040E050E0CE010E94BE2F809133
:105BA000E8008E778093E80080E2FE01ACE2B5E089
:105BB00001900D928A95E1F7DF91CF91089580933E
:105BC000290570932B0560932A058091D3068430B4
:105BD00001F582E08093E9008FEF9091E800815019
:105BE00095FD06C095ED9A95F1F700008111F5CF6E
:105BF0008091E80085FF0DC040E050E063E070E078
:105C000089E295E00E94BE2F8091E8008E77809314
:105C1000E8000895BC0184E00C94DF2DBC0183E012
:105C20000C94DF2D8091D206811109C00E944F3162
:105C30000E94AC318091E20084608093E20008957C
:105C40001092D20608950C946A2C6091CF0681E0E0
:105C5000611101C080E00C94552C9091D30681E035
:105C6000943009F080E06091CF060C945A2C42E009
:105C700061EC81E00E94C83042E261EC82E00E9467
:105C8000C8309091D30681E0943009F080E06091B3
:105C9000CF060C94632C8091D506833009F461C043
:105CA00030F4813071F0823009F49AC008958A305E
:105CB00009F486C08B3009F46CC0893009F0A8C0A3
:105CC00020C08091D406813A09F0A2C08091E800FA
:105CD000877F8093E8008091D8069091D906892B20
:105CE00021F460E28CE295E003C060E080E090E0A7
:105CF00070E00E9409308091E8008B778093E80083
:105D000008958091D406813209F082C08091D8062E
:105D10009091D906029708F07BC08091E800877FB8
:105D20008093E8008091E80082FD05C08091D30651
:105D30008111F8CF6DC02091F3008091F20090E0C6
:105D4000922B029731F48091F100813011F086306E
:105D500021F48091F10080934C058091E8008B77CD
:105D600053C08091D406813A09F052C08091D80680
:105D70009091D906892B09F04BC08091E800877F6C
:105D80008093E8008091E80080FFFCCF80913B0287
:105D900036C08091D4068132D9F58091D806909191
:105DA000D906892BA9F58091E800877F8093E800C8
:105DB0000E94FD308091D60680933B020C9494079C
:105DC0008091D406813221F58091E800877F80930D
:105DD000E8000E94FD308091D70680934D0508951C
:105DE0008091D406813AA1F48091E800877F809366
:105DF000E8008091E80080FFFCCF80914D05809302
:105E0000F1008091E8008E778093E8000C94FD30DB
:105E1000089584B7877F84BF0FB6F894A8958091C2
:105E20006000886180936000109260000FBE90E077
:105E300080E80FB6F89480936100909361000FBEE4
:105E40000C94652C0E944F310E94AC31E2EEF0E0E0
:105E500080818460808378940C9441348FE292E056
:105E60000C942C2B8091D3068530A9F48091D30615
:105E7000853079F40E94B62C8091D1068823B1F345
:105E80000E94772C882391F30E94A82F0E949407E8
:105E9000EDCF0C94E12C089508950C944F2F292FE9
:105EA000332723303105C9F060F42130310581F00A
:105EB0002230310509F044C08BE390E02AE334E05E
:105EC00043C021323105E1F02232310549F138C0B9
:105ED00082E190E025E734E037C0992781309105D1
:105EE00049F028F0029761F5E4E1F4E005C0E6E34B
:105EF000F4E002C0E6E2F4E0849190E09F0124C067
:105F00006115710541F061307105D1F489E090E0CF
:105F100025E634E019C089E090E02CE434E014C0B8
:105F20006115710541F06130710551F486EB90E027
:105F300027E834E009C080E490E02DE335E004C0B8
:105F400080E090E020E030E0FA0131832083089582
:105F500080E189BD82E189BD09B400FEFDCF809159
:105F6000D8008F7D8093D8008091E000826080937C
:105F7000E0008091E00081FDFCCF0895CF92DF9298
:105F8000EF92FF920F931F93CF93DF93EC018B015E
:105F90007A010E941C31811133C0E114F10439F0FF
:105FA000F70180819181081B190BC80FD91FC12CE3
:105FB000D12C0115110519F18091E80085FD16C05D
:105FC0008091E8008E778093E800E114F10449F0B5
:105FD000F70180819181C80ED91ED182C08285E0EF
:105FE0000FC00E941C31882321F30AC0899180933D
:105FF000F10001501109FFEFCF1ADF0ADACF80E07C
:10600000DF91CF911F910F91FF90EF90DF90CF9094
:1060100008952091DA063091DB062617370748F0FD
:106020006115710539F42091E8002E772093E8007E
:1060300001C0B901FC0120E06115710579F1809181
:10604000D3068823F1F18530F1F18091E80083FDDA
:106050003CC08091E80082FD2EC08091E80080FF66
:10606000EBCF2091F3008091F20090E0922B61152C
:10607000710551F08830910538F421912093F10099
:10608000615071090196F3CF21E0089709F020E0F3
:106090008091E8008E778093E800CECF2111CFCF9A
:1060A0000AC08091D306882361F0853061F0809129
:1060B000E80083FD0AC08091E80082FFF2CF80E013
:1060C000089582E0089583E0089581E00895209185
:1060D000DA063091DB062617370748F0611571059F
:1060E00039F42091E8002E772093E80001C0B9012F
:1060F000FC0120E06115710591F18091D3068823A0
:1061000009F440C0853009F43FC08091E80083FD68
:106110003DC08091E80082FD2FC08091E80080FFA3
:10612000E9CF2091F3008091F20090E0922B61156D
:10613000710559F08830910540F424912093F100C5
:106140003196615071090196F2CF21E0089709F06C
:1061500020E08091E8008E778093E800CBCF21117A
:10616000CCCF0AC08091D306882361F0853061F0DE
:106170008091E80083FD0AC08091E80082FFF2CFA1
:1061800080E0089582E0089583E0089581E0089515
:10619000982F973068F59093E900981739F070912F
:1061A000EC002091ED005091F00003C0242F762FD9
:1061B00050E021FD02C09F5FECCF3091EB003E7FAD
:1061C0003093EB003091ED003D7F3093ED00309146
:1061D000EB0031603093EB007093EC002093ED0006
:1061E0005093F0002091EE0027FDE5CF80E0089568
:1061F0008F708093E90081E008958091D40687FF35
:1062000011C08091E80082FD05C08091D306811104
:10621000F8CF11C08091E8008B770BC08091D30636
:10622000882349F08091E80080FFF8CF8091E80052
:106230008E778093E80008952091E4003091E50086
:1062400095E64091EC00842F817040FF23C080913F
:10625000E80080FD1DC08091D306882399F0853029
:1062600099F08091EB0085FD11C04091E4005091C0
:10627000E5002417350729F3915011F09A01E1CF79
:1062800084E0089582E0089583E0089581E0089510
:1062900080E008954091E80042FFDDCF08950E941C
:1062A000BD310E94C531E0EEF0E0808181608083E5
:1062B000E8EDF0E080818F77808319BCA7EDB0E036
:1062C0008C918E7F8C9380818F7E80831092D206FA
:1062D00008950F931F93CF93DF930E94BD310E94C7
:1062E000C531C8EDD0E088818F7788838881806848
:1062F000888388818F7D888319BC1092D306109281
:10630000CF061092D1061092D00600EE10E0F801F0
:1063100080818B7F808388818160888342E060E018
:1063200080E00E94C830E1EEF0E080818E7F8083C3
:10633000E2EEF0E0808181608083808188608083EC
:10634000F80180818E7F8083888180618883DF91DE
:10635000CF911F910F910895E8EDF0E080818F7E3D
:106360008083E7EDF0E080818160808384E082BFFC
:1063700081E08093D2060C946931E8EDF0E08081F1
:106380008E7F80831092E20008951092DA001092BE
:10639000E10008951F920F920FB60F9211242F93D0
:1063A0003F934F935F936F937F938F939F93AF939D
:1063B000BF93EF93FF938091E10082FF0BC0809128
:1063C000E20082FF07C08091E1008B7F8093E100B3
:1063D0000E9440348091DA0080FF1FC08091D80075
:1063E00080FF1BC08091DA008E7F8093DA0080915D
:1063F000D90080FF0DC080E189BD82E189BD09B46B
:1064000000FEFDCF81E08093D3060E94122E05C0CE
:1064100019BC1092D3060E94202E8091E10080FFCB
:1064200019C08091E20080FF15C08091E2008E7F4C
:106430008093E2008091E20080618093E20080918D
:10644000D80080628093D80019BC85E08093D30681
:106450000E94252E8091E10084FF30C08091E200EF
:1064600084FF2CC080E189BD82E189BD09B400FEB2
:10647000FDCF8091D8008F7D8093D8008091E1007E
:106480008F7E8093E1008091E2008F7E8093E20016
:106490008091E20081608093E2008091CF068823A2
:1064A00011F084E007C08091E30087FD02C081E025
:1064B00001C083E08093D3060E942D2E8091E100DD
:1064C00083FF29C08091E20083FF25C08091E10015
:1064D000877F8093E10082E08093D3061092CF06FD
:1064E0008091E1008E7F8093E1008091E2008E7FB9
:1064F0008093E2008091E20080618093E20042E0BC
:1065000060E080E00E94C8308091F0008860809355
:10651000F0000E94232EFF91EF91BF91AF919F91C8
:106520008F917F916F915F914F913F912F910F903C
:106530000FBE0F901F9018951F920F920FB60F92DB
:1065400011242F933F934F935F936F937F938F9378
:106550009F93AF93BF93CF93DF93EF93FF93C0913C
:10656000E900CF708091EC00D82FD17080FDD0E889
:106570001092E9008091F000877F8093F00078947A
:106580000E94E0321092E9008091F00088608093D0
:10659000F000CD2BCF70C093E900FF91EF91DF9118
:1065A000CF91BF91AF919F918F917F916F915F91AB
:1065B0004F913F912F910F900FBE0F901F90189504
:1065C0001F93CF93DF93CDB7DEB7AA970FB6F8949A
:1065D000DEBF0FBECDBFE4EDF6E08091F100819308
:1065E00026E0EC3DF207C9F70E944B2E8091E800AF
:1065F00083FF2EC18091D4069091D506492F50E09B
:106600004A30510508F024C1FA01EE59FF4F0C94AD
:10661000C534803821F0823809F01AC108C0809151
:10662000D0069091D106992389F082600FC08091A5
:10663000D8068F70873008F00BC18093E9008091F5
:10664000EB0085FB882780F91092E9009091E80023
:10665000977F9093E8008093F1001092F100D1C0F1
:10666000282F2D7F09F0F4C0882319F0823061F0C3
:10667000EFC08091D606813009F0EAC0933009F06E
:1066800080E08093D1062EC08091D60681112AC069
:106690008091D8068F702FEF280F263008F0D8C0D1
:1066A0008093E9002091EB0020FF1CC0933021F47F
:1066B0008091EB00806214C09091EB009061909308
:1066C000EB0021E030E0A90102C0440F551F8A957C
:1066D000E2F74093EA001092EA008091EB008860B4
:1066E0008093EB001092E9008091E800877F80930F
:1066F000E8000E94FD30ACC08111AAC01091D606FE
:106700001F778091E3008078812B8093E300809154
:10671000E800877F8093E8000E94FD308091E800C8
:1067200080FFFCCF8091E30080688093E30011112B
:1067300002C082E001C083E08093D30689C0805804
:10674000823008F085C08091D6069091D7068C3DA6
:1067500053E0950779F583E08A838AE289834FB70E
:10676000F894DE01139620E03EE051E2E32FF0E0E2
:1067700050935700E49120FF03C0E295EF703F5F14
:10678000EF708E2F90E0EA3010F0C79601C0C096EF
:106790008D939D932F5F243149F74FBF8091E8007F
:1067A000877F8093E8006AE270E0CE0101960E9444
:1067B000093016C06091D8067091D906AE014F5FBE
:1067C0005F4F0E944D2FBC01892B09F441C090916D
:1067D000E800977F9093E80089819A810E94673052
:1067E0008091E8008B778093E80032C0803881F593
:1067F0008091E800877F8093E8008091CF068093A6
:10680000F1008091E8008E7772CF811121C08091D4
:10681000D6069091D70699270297D4F48091E80084
:10682000877F8093E8008091D6068093CF060E94F0
:10683000FD308091CF06811106C08091E30087FD75
:1068400002C081E001C084E08093D3060E94372E0D
:106850008091E80083FF0AC08091E800877F8093E1
:10686000E8008091EB0080628093EB00AA960FB65F
:10687000F894DEBF0FBECDBFDF91CF911F91089579
:106880000895CF938091D3068823A1F0C091E900A9
:10689000CF709091EC00892F817090FD80E8C82B1B
:1068A0001092E9008091E80083FD0E94E032CF70F1
:1068B000C093E900CF910895AA1BBB1B51E107C00B
:1068C000AA1FBB1FA617B70710F0A61BB70B881F80
:1068D000991F5A95A9F780959095BC01CD0108950F
:1068E00097FB072E16F4009407D077FD09D00E947D
:1068F0005C3407FC05D03EF4909581959F4F089538
:10690000709561957F4F0895A1E21A2EAA1BBB1BBB
:10691000FD010DC0AA1FBB1FEE1FFF1FA217B3076B
:10692000E407F50720F0A21BB30BE40BF50B661F81
:10693000771F881F991F1A9469F760957095809545
:1069400090959B01AC01BD01CF010895052E97FBE9
:106950001EF400940E94BD3457FD07D00E94843479
:1069600007FC03D04EF40C94BD34509540953095FF
:1069700021953F4F4F4F5F4F0895909580957095AB
:1069800061957F4F8F4F9F4F0895EE0FFF1F05902A
:10699000F491E02D09948F929F92AF92BF92CF9283
:1069A000DF92EF92FF92CF93DF93EC0168817981C0
:1069B0008A819B81611571058105910521F464E24D
:1069C00079ED8BE597E02DE133EF41E050E00E9457
:1069D000A63449015A019B01AC01A7EAB1E40E9427
:1069E00098356B017C01ACEEB4EFA50194010E94D7
:1069F000A635DC01CB018C0D9D1DAE1DBF1DB7FF63
:106A000003C00197A109B04888839983AA83BB83F7
:106A10009F77DF91CF91FF90EF90DF90CF90BF9065
:106A2000AF909F908F9008950E94CB34089580E09E
:106A300091E00E94CB340895A0E0B0E08093000183
:106A400090930101A0930201B09303010895FB010B
:106A5000DC0102C005900D9241505040D8F70895D6
:106A6000FB01DC0104C08D910190801921F441509B
:106A70005040C8F7881B990B0895FB01DC0102C048
:106A800001900D9241505040D8F70895DC01CB01A0
:106A9000FC01F999FECF06C0F2BDE1BDF89A31962E
:106AA00000B40D9241505040B8F70895F999FECFC7
:106AB00092BD81BDF89A992780B50895A8E1B0E00C
:106AC00042E050E00C944835DC01A40FB51F415062
:106AD000504048F0CB01840F951F2E910E947535D0
:106AE00041505040D0F70895262FF999FECF92BD1E
:106AF00081BDF89A019700B4021639F01FBA20BD83
:106B00000FB6F894FA9AF99A0FBE08950396272FB4
:106B10000E9475350E947435252F0E947535242FEB
:106B20000C9475350196272F0E9475350C94743599
:106B30000E94AB35A59F900DB49F900DA49F800D32
:106B4000911D11240895B7FF0C9498350E94983533
:106B5000821B930B0895A29FB001B39FC001A39F16
:106B6000700D811D1124911DB29F700D811D112486
:086B7000911D0895F894FFCF78
:106B780001000000000102030405060708090A0BCA
:106B88000C0D0E0F101112131415161718191A1BC5
:106B98001C1D1E1F20212223242526272829FF2AE1
:106BA8002B2C2D2E2F3031323334353637FF3839F0
:106BB8003A3B3CFFFF3DFFFF3E3F4041FF42430061
:106BC800000F001E002D003C004B005A00690078A1
:106BD8000087009600A500B400CB00E00004101761
:106BE8001026103510441053106210711080108F49
:106BF800109E10AD10BC10CE10E01006201A2029EF
:106C0800203820472056206520742083209220A118
:106C180020B020C920E02009302230313040304FE8
:106C2800305E306D307C308B309A30A930BD30D238
:106C380030E03002401540274060409640A540B4FF
:106C480040C340D240E040010404040404040404A6
:106C580004040404040101040404040404040404F2
:106C680004040404010104040404040404040404E2
:106C780004040101040404040404040404040404D2
:106C88000101010104010101010101C8005E03289D
:106C98000850011E0A14010300FF00FFFF39057B9D
:106CA8002D9E2D7F2D0E2E0A2E7E2D0100FFC8E26F
:106CB80000E900EA00B500B600B700CD008301CCBA
:106CC800008A01920194012102230224022502264E
:106CD8000227022A02B300B4006F00700081828389
:106CE800E200E900EA00B500B600B700CD00830174
:106CF800CC008A0192019401210223022402250278
:106D0800260227022A02B300B4006F0070008182B5
:106D180083F7F6F56730313233349796949593922A
:106D2800F0F1F4C666003131295A1B750A2425C1D1
:066D38002508261C2500C1
:00000001FF
